:046F2B00010001431D
:10699D00AF50055074D02FF582E4341DF583E59981
:1069AD00F022D3E5309400E52F94002290000FE003
:0369BD006403224E
:030003000256A7FB
:0B56A700C0E0C083C082C0D075D008F6
:1056B200852E82852D83E493FF201404C4540FFFAA
:1056C200430FF08F80C284D28500C2870000D28748
:1056D200007580FF7580FEC284C28500C28700000B
:1056E200D287007580FF30140CC214052EE52E708F
:0956F20006052D8002D214D2A895
:0956FB00D0D0D082D083D0E0327F
:03000B0002197B5C
:10197B00C0E0C0F0C083C082C0D075D008758CD8D1
:10198B00758A92D28C1242271262F1E531D3940000
:10199B0040171531E53164056009E531640F6003CB
:1019AB00021B8D126BE2021B8D753114E54ED39425
:1019BB00004002154EE54FD394004002154FE53A17
:1019CB00D394004002153AE54BD394004002154BDB
:1019DB00154CE54C123A601B7F001B54011B2C026B
:1019EB001B04031A81041A68051A4F061A36071AC4
:1019FB001D081A040900001B8AD3E52C9400E52B63
:101A0B0094005003021B8DE52C152C704D152B02E9
:101A1B001B8DD3E5379400E53694005003021B8DE4
:101A2B00E537153770021536021B8DD3E548940048
:101A3B00E54794005003021B8DE5481548700215CD
:101A4B0047021B8DD3E54A9400E5499400500302ED
:101A5B001B8DE54A154A70021549021B8DD3E52AE9
:101A6B009400E52994005003021B8DE52A152A707A
:101A7B00021529021B8D7885E6FF7003021B8DEF83
:101A8B00B40105900524801BEFB402101269AF401E
:101A9B002FE53015307002152F021B8DEFB4030CA0
:101AAB00900526E0F52FA3E0F5308028EFB4041263
:101ABB001269AF400BE53015307002152F021B8DEC
:101ACB008012EF64057003021B8DEFB4060C752FAB
:101ADB0002753058788506021B8DEF640760030290
:101AEB001B8D1269AF400BE53015307002152F02BC
:101AFB001B8D78857600021B8DD3E5399400E53874
:101B0B0094004008E539153970021538D3E53C943B
:101B1B0000E53B9400406BE53C153C7002153B80A7
:101B2B0061D3E5579400E55694004008E5571557E7
:101B3B0070021556D3E5559400E55494004043E5E7
:101B4B00551555700215548039D3E5359400E5349D
:101B5B0094004008E535153570021534301523D344
:101B6B00E5339400E53294004018E53315337012D9
:101B7B001532800EE551D394004004155180007549
:0D1B8B004C0AD0D0D082D083D0F0D0E03210
:03001300023EF5B5
:0D3EF500C0E0C0F0C083C082C0D075D01006
:103F0200E545C394504003023FB6202403023FB666
:103F1200300C03023FB6E5A0540FF5587D077F0130
:103F2200124EE95067202364E545700DE558B40C44
:103F320008201105D211023FB620034A2011471270
:103F42003FC150047F0180027F0F126EAE90000FBE
:103F5200E0FF64016012EFB40302800C90000FE0F6
:103F6200B40209123FC150047F80801290000FE01A
:103F7200B4020E7D037F07124EE940057FA01200B6
:103F820016754202D20390053CE0F53A90002BE010
:103F9200B5580D7D087F05124EE95004D2268014D3
:103FA200053EE53EAE3D7002053D14F5828E83E589
:043FB20058F0054579
:103FB600D0D0D082D083D0F0D0E0327D037F0712FC
:033FC6004EE9229F
:030023000263CAAB
:1063CA00C0E0C083C082C0D075D018309819C29876
:1063DA00E599B40A0812699D755000800AE550C310
:1063EA009490500312699D309902C299D0D0D082FC
:0563FA00D083D0E03269
:03003B0002493443
:0D493400C0E0C0F0C083C082C0D075D018B4
:10494100C2CEE546C39410507C302579200C76AF59
:10495100A07804EF08800123D8FDF55953590F7D44
:10496100077F02124EE95035202332E546700CE5EF
:1049710059B40C07201304D213804A2004192013C0
:104981001690000FE0B4020F7F0A126EAE7F801204
:104991000016754202D20490053CE0F53A90002BD6
:1049A100E0B5590D7D087F05124EE95004D22880EB
:1049B100140540E540AE3F7002053F14F5828E8339
:0549C100E559F0054678
:0B49C600D0D0D082D083D0F0D0E032FF
:104B9300E4F55AF55B755C1E755DFF855B82855A8E
:104BA30083E0F55E635EFFE55EF0E0655E60031241
:104BB3006F2F635EFF855B82855A83E55EF0E06558
:104BC3005E6003126F2F055BE55B7002055AE55DBE
:104BD300155D7002155CD3E55D9400E55C940050AF
:104BE300BA75985A758921758845758DE7758780DB
:104BF300758CD8758AEF75C90275C808753D1E7521
:104C03003E60753F1E7540B075B701D2A9D2E8D298
:0F4C1300AA75C64C75EEFF75FEFFD2AF12669AFA
:014C2200226F
:026F2F0080FEE2
:10697A00202F0F90053AE0F54EE54ED394004012D1
:10698A0080F7302F0D90053AE0F54FE54FD394008C
:03699A0050F9228F
:1069320030310AD215900024E04420800DC2157F28
:1069420008126EEF900024E054DFF0FD7F247E00F9
:046952001263942216
:102ED2008F70E570640170292030047F01805620D4
:102EE2003003022FCD122FDE4003022FCD122FE628
:102EF200500C122FCE301503022FCD022FC3022FFA
:102F020083E570640270202030047F028027203025
:102F120003022FCD122FEE4003022FCD1269B9709A
:102F220003022FCD022F9DE57064036003022FCDB3
:102F32002030057F03026EEF303024122FDE501F47
:102F4200122FEE501A1269B96015122FE6500B7F3C
:102F52000A122FF6201574022FC37F03022FCA30E4
:102F62003023123004501E7D017F02124EE94015BB
:102F72007D017F07124EE95008122FCE20154C809A
:102F8200407F01804330301712300440127D017FB0
:102F920002124EE950091269B960047F0280293099
:102FA20030297D017F01124EE950201269B9701B50
:102FB2007D017F07124EE9500D7F09122FF6201571
:102FC2000AD2310269327F01126F02227F09126F27
:102FD20002900536E0F532A3E0F533227D017F0150
:102FE200124EE9227D017F07124EE9227D017F0206
:102FF200124EE922126F02900536E0F532A3E0F597
:0A30020033227D017F01124EE92206
:104C2300C2957FFF126EEF124B937F0712632850DA
:104C33000512003E8003126074D28C7F0812632831
:104C430050051242E780FEC22B1268539000D1E058
:104C5300FF7C117D00125BEF125D6290000FE0B4E8
:104C63000105122839801090000FE0FF64026004F0
:104C7300EFB4030312326D123D34301E11E542705E
:104C83000DE52754A060077FA0126EAEC21E7D07FC
:104C93007F05124EE94002C200E552C3940A50BB9D
:104CA3003015B8E533453270B2C23112693280AB88
:104A6A00EF253EFFEE353DCF2401FDE43FFC22AFAA
:104A7A005A7E00EF2403FDEE33FC22E53E255AF56B
:104A8A0082E4353DF58322E540255AF582E4353F37
:104A9A00F58322E56F256DF582E4356EF583E0FF37
:104AAA00E56F256DF582E4356EF58322E55A240219
:104ABA00FFE433FE22E56C2401FFE433FEC3E56D17
:104ACA009FEE6480F874809822EF2540FFEE353F10
:104ADA0022C2017FF47E01126C38E56C25E0F56C88
:104AEA00756D0122E55C2EF582E4355BF583E0FD08
:084AFA0022753D1E753E60228D
:106C3800EF1FAA0670011ED39400EA9400400BE4EB
:0A6C4800FDEDC394C850E90D80F77C
:016C5200221F
:105180008F5BE55BB401197D017F06124EE9500C7F
:105190009000B1E0FF7C0D7D00125BEF7885062268
:1051A000E55BB402131251F250439000B2E0FF7C71
:1051B0000D7D20125BEF8035E55BB404161251F2D1
:1051C000500C9000B4E0FF7C0D7D60125BEF7885A1
:1051D000760622E55BB403197D027F06124EE95084
:1051E0000C9000B3E0FF7C0D7D40125BEF7885767C
:0A51F00001227D027F06124EE92223
:104EE900BF0107900020E0FE8048BF020790002123
:104EF900E0FE803EBF0307900022E0FE8034BF043D
:104F090007900023E0FE802ABF0507900024E0FEF9
:104F19008020BF0607900025E0FE8016BF07079096
:104F29000026E0FE800CBF0807900027E0FE800203
:104F3900E4FEBD0103EE1322BD0204EEA2E122BD8F
:104F49000304EEA2E222BD0404EEA2E322BD05049D
:104F5900EEA2E422BD0604EEA2E522BD0704EEA2FC
:074F6900E622BD0802EE3351
:014F7000221E
:101D9900124AFB900100E0F55A124A85E0123A60B6
:101DA9001DC8011DFD021E32031E67041E9C051E6F
:101DB900D1061F06071F36081F620900001F8C1273
:101DC9004A85A3E0B40A15E55A124AB8E545B507AC
:101DD9000BE4B506077D017F01021F4A124A79E526
:101DE900456D7001EC6003021F8C124A6AC2297F9B
:101DF90001021F5F124A85A3E0B40A15E55A124A87
:101E0900B8E545B5070BE4B506077D017F02021F5A
:101E19004A124A79E5456D7001EC6003021F8C1284
:101E29004A6AC2297F02021F5F124A85A3E0B40AE7
:101E390015E55A124AB8E545B5070BE4B506077D1D
:101E4900017F03021F4A124A79E5456D7001EC6072
:101E590003021F8C124A6AC2297F03021F5F124ABA
:101E690085A3E0B40A15E55A124AB8E545B5070B4A
:101E7900E4B506077D017F04021F4A124A79E54548
:101E89006D7001EC6003021F8C124A6AC2297F043B
:101E9900021F5F124A85A3E0B40A15E55A124AB82F
:101EA900E545B5070BE4B506077D017F05021F4A25
:101EB900124A79E5456D7001EC6003021F8C124AE4
:101EC9006AC2297F05021F5F124A85A3E0B40A1579
:101ED900E55A124AB8E545B5070BE4B506077D0191
:101EE9007F06021F4A124A79E5456D7001EC6003CD
:101EF900021F8C124A6AC2297F06021F5F124A8595
:101F0900A3E0B40A14E55A124AB8E545B5070AE44C
:101F1900B506067D017F078028124A79E5456D706F
:101F290001EC705F124A6AC2297F078029124A852B
:101F3900A3E0B40A0F124A85A3A3E070077D017FCD
:101F490008024E5E124A79E5456D7001EC70341253
:101F59004A6AC2297F08021014124A85A3A3E070B5
:101F690022124A85A3E024F96008147016E4FF02DE
:101F79005EFE7FF47E01126C387D5E7F0212667010
:031F89001242E71A
:011F8C002232
:101B9800753F1E7540B0900108E0F55A124A91E071
:101BA800123A601BCA011C02021C3A031C72041C74
:101BB800AA051CE2061D1A071D4D081D8209000012
:101BC8001D98124A91A3E0B40A13124AB6E546B525
:101BD800070BE4B506077D017F01021D65AF5A12A8
:101BE8004A7BE5466D7001EC6003021D98124AD3EA
:101BF800124A71D2297F01021D7F124A91A3E0B4D3
:101C08000A13124AB6E546B5070BE4B506077D0187
:101C18007F02021D65AF5A124A7BE5466D7001ECE2
:101C28006003021D98124AD3124A71D2297F020218
:101C38001D7F124A91A3E0B40A13124AB6E546B5CD
:101C4800070BE4B506077D017F03021D65AF5A1235
:101C58004A7BE5466D7001EC6003021D98124AD379
:101C6800124A71D2297F03021D7F124A91A3E0B460
:101C78000A13124AB6E546B5070BE4B506077D0117
:101C88007F04021D65AF5A124A7BE5466D7001EC70
:101C98006003021D98124AD3124A71D2297F0402A6
:101CA8001D7F124A91A3E0B40A13124AB6E546B55D
:101CB800070BE4B506077D017F05021D65AF5A12C3
:101CC8004A7BE5466D7001EC6003021D98124AD309
:101CD800124A71D2297F05021D7F124A91A3E0B4EE
:101CE8000A13124AB6E546B5070BE4B506077D01A7
:101CF8007F06021D65AF5A124A7BE5466D7001ECFE
:101D08006003021D98124AD3124A71D2297F060233
:101D18001D7F124A91A3E0B40A12124AB6E546B5ED
:101D2800070AE4B506067D017F078031AF5A124ADB
:101D38007BE5466D7001EC7057124AD3124A71D296
:101D4800297F078032124A91A3E0B40A13124AB6D7
:101D5800E546B5070BE4B506077D017F08024E5E30
:101D6800AF5A124A7BE5466D7001EC7023124AD3D4
:101D7800124A71D2297F08021014124A91A3A3E0D3
:101D8800700E124A91A3E024F870057F01125EFEDE
:011D98002228
:0447E7008C5B8D5CFE
:1047EB00055CE55C7002055B14F5828C83E0F97067
:1047FB000302488EEF7005124AFB8009BF01067554
:10480B003F1E7540B0302946EF7007E965456002E1
:10481B00C322BF0107E965466002C322E4FEEEC373
:10482B00995029EF700F124AEEE53E2E124A89E09D
:10483B006D6002C322EF6401700F124AEEE5402E49
:10484B00124A95E06D6002C3220E80D2D32220293A
:10485B0033E4FEEEC3995029EF700F124AEEE53E9A
:10486B002E124A89E06D6016C322EF6401700F129D
:10487B004AEEE5402E124A95E06D6002C3220E808F
:04488B00D2D322C39F
:01488F002206
:061014008F5BAB05AA048E
:10101A007D027F07124EE95011E55BB4050C8B8205
:10102A008A83E0640570030212817D017F07124EF4
:10103A00E95011E55BB4050C8B828A83E064067083
:10104A0003021281C22AEB24FFF582EA34FFF583F8
:10105A00E0F55D8B828A83E0FFF55EA3E0F9F55F38
:10106A00EF123A60108A01109102109803109F043F
:10107A0010A60510AD0610B40710BB08000010C07A
:10108A00755C01D22A802F755C02D22A8028755C91
:10109A0004D22A8021755C08D22A801A755C10D283
:1010AA002A8013755C20D22A800C755C40D22A8073
:1010BA0005755C80D22AE924FE700302118224F8A5
:1010CA00605C24096003021194E55BB40105900099
:1010DA00208045E55BB40205900021803BE55BB4C6
:1010EA0003059000228031E55BB40405900023805B
:1010FA0027E55BB40505900024801DE55BB4060571
:10110A009000258013E55BB407059000268009E569
:10111A005B64087077900027E0455CF0806EE55BC1
:10112A00B401059000208045E55BB40205900021DA
:10113A00803BE55BB403059000228031E55BB40493
:10114A00059000238027E55BB40505900024801DE7
:10115A00E55BB406059000258013E55BB4070590AE
:10116A0000268009E55B64087022900027E0FFE50D
:10117A005CF4FEEF5EF08014E55BB4050D8B828AA9
:10118A0083E0FFD22F12299AC22AC22A202A0302F6
:10119A001281E55BB40109900020E0FD7F208060A8
:1011AA00E55BB40209900021E0FD7F218052E55BF6
:1011BA00B40309900022E0FD7F228044E55BB40479
:1011CA0009900023E0FD7F238036E55BB405099092
:1011DA000024E0FD7F248028E55BB4060990002501
:1011EA00E0FD7F25801AE55BB40709900026E0FD43
:1011FA007F26800CE55BB4080C900027E0FD7F2772
:10120A007E00126394126D4DD2AF2029047F0180B3
:10121A00027F02126F02A229922F12697AAD5DE44F
:10122A00FF126670AD5EE4FF126670E55FB40104FA
:10123A007D388007E55FB40A077D367F061266703F
:10124A00E55BB405031264F87D077F05124EE95089
:10125A000A200007C2307F03122ED27D017F0112BD
:10126A004EE94005C230122ED27D017F02124EE9AC
:07127A004005C230122ED224
:01128100224A
:024E5E008F5B68
:104E6000ED24FF922F12697AE55B123A604E8901B8
:104E70004E8E024E93034E98044E9D054EA2064E52
:104E8000A7074EAC0800004EB29000208021900091
:104E900021801C9000228017900023801290002413
:104EA000800D90002580089000268003900027E068
:104EB000F55CE55C6024755E01E4F55DE55C30E081
:104EC00007AD5EE4FF126670E55CC313F55C055E3A
:104ED000055DE55DC3940840E3227D187F021266FC
:084EE000707D537F0212667021
:014EE80022A7
:10632800C2AFD284C285BF070BC28600E580A2E255
:10633800922A8019BF080BC28600E580A2E3922A40
:10634800800BBF0508C28600E58013922AD286D248
:0563580085D2AFA22A6E
:01635D00221D
:10468700C229D22DE4FF1259D07D2E7F0312667006
:104697007D607F021266707F03126EEF3024FD206B
:1046A70024FDE5456407703B7E017F50124AFB8F6E
:1046B700828E837407F07D01E53E2D124A89E582DB
:1046C70024FFF582E58334FFF583E0F9EF2DF582CA
:1046D700E43EF583E9F00DBD08DED2297F647E0054
:1046E700126C387F081263285043302995D22DE485
:1046F700FF1259D07D607F021266707D327F0612ED
:1047070066707D1E7F05126670C22DE4FF1259D0B8
:104717007C017D507B087F507E0112551C7F08125B
:10472700632850097F327E00126C3880F07F647EE8
:0447370000126C38C8
:01473B00225B
:0254B3008F5A0E
:1054B500900138E0F55BE55A7020E55B124AB8E5E6
:1054C500456F7001EE704F7460255BF582E4341E04
:1054D500AF82F55D8F5E7F408024E55A64017036AA
:1054E500E55B124AB8E5466F7001EE702974B02588
:1054F5005BF582E4341EAF82F55D8F5E7F1012008E
:1055050016855E82855D83E0FFA3E0FD126D9B8FAE
:065515005CE4FD124F7181
:01551B00226D
:024F71008D6B46
:104F730075F020EF900280123A54AF8285836E8FD2
:104F83006FE0F56CD394004060E56C9410505AE5E3
:104F93006B7014124ADD124ABF504E124A9D124FD3
:104FA300F2056D056D80EFE56B64017019124ADB44
:104FB300124ABF5034124A9D124FF2302402802904
:104FC300056D056D80EAE56B6402701D124ADB1204
:104FD3004ABF5015124A9DA3E0FD126528302403F1
:0E4FE300024D42056D056D80E67F50126EAEE8
:084FF10022A3E0FD1265282255
:100A5400855C82855B83A3A3E0FF855C82855B83E1
:100A6400A3222430F58274003EF583EDF0AF62EFEB
:100A74003395E0FEE55F2FF582E55E3EF583A3A3A3
:100A8400E0FF126D76AD07AF63EF3395E0FEEF2222
:100A9400A3A3E0FFE55C2404F582E4355BF583E081
:100AA40022E55F2405F582E4355EF583E022E55F07
:100AB4002405F582E4355EF583E0FFE55F2406F561
:100AC40082E4355EF583E0222431F58274003EF53C
:100AD40083EDF0AF62EF3395E0FEE55F2FF582E53D
:100AE4005E3EF583222455F582E4340AF583EFF063
:100AF400E56275F007A422E562FD3395E0FCE55F4D
:100B04002DF582E55E3CF583E0FFE55F2DF582E59A
:100B14005E3CF58322AF60EF3395E0FEE56175F04E
:100B240008900158123A54E5822FF582E5833EF588
:100B340083228E69F56AAF68EF3395E0FEE5662F90
:100B4400F582E5653EF58322A3A3A3E0FF8D828CA5
:100B540083E5822404F582E43583F58322E5662463
:100B640005F582E43565F583E022E55E75F007A4BA
:100B74002454F582E4340AF58322E55E75F007A473
:100B84002451F582E4340AF5832224E0F582740AC0
:100B94003EF583E5822DF582E5833CF58322E55E0F
:100BA40075F007A42453F582E4340AF58322E55F43
:100BB4002405F582E4355EF583E0FFE55F2406F560
:100BC40082E4355EF583E022E55E75F007A42452E5
:100BD400F582E4340AF58322749F2562F582E434B5
:100BE40000F58322746F2562F582E43400F58322D4
:100BF4002450F582E4340AF58322ECFF3395E0FEB9
:100C0400EF25E0FFEE33FE75F02022E5602405F5C4
:100C140082E4355FF58322D3EF6480948022AB07AE
:100C2400AA068B828A83A3A3A3E0FFEB2404F582A4
:100C3400E43AF583E0FD228F828E83A3A3A3E0220E
:100C4400855F82855E83A3A322AB5DAD5AAF5CAEA4
:100C54005B2233CE33CE92E022A2E0CE13CE132217
:100C640075F00AA42DFDE5F03CFCE56622E5602460
:100C740005F582E4355FF583E022E56275F00890BE
:100C84000158023A54E55E75F007A42455F582E450
:100C9400340AF583E022AB5AAD5DAF5CAE5B22EF64
:100CA4007C002563FDEC35628D82F58322A3A3E0ED
:100CB400FFAD5A22E5662DF582E5653CF583A3A3D5
:100CC40022540FF5657808AF03AE02EF08220564DD
:100CD400E564AE632275F020123A54E0FEA3E0FF0F
:100CE40022E0FAA3E0FB780CFFAE020822E0FCA3AA
:100CF400E0FD7804FFAE040822E5632561F582E493
:100D04003562F58322E5662DF582E5653CF583229F
:100D1400E5662FF582E5653EF583222480F582742D
:100D2400023EAF82222560F560E4355FF55F2285DF
:100D34006082855F83228F828E83A3A3E0640A226C
:02055B008F5AB5
:10055D00C22AE4F542D223D22D1259D07D4B7F020F
:10056D001266707D02E4FF1266707D32E4FF126642
:10057D00707D607F021266707D027F07124EE9501A
:10058D00057F04126EEF900528E0F536A3E0F537F0
:10059D007F03126EEFE55A7006A22492298009E5B9
:1005AD005AB40104A2259229E53745367005D22AA1
:1005BD00020A223029DFE55A7006A2249229800909
:1005CD00E55AB40104A22592292029EAE55A700BB7
:1005DD00755B1E755C6085455D800EE55AB401093D
:1005ED00755B1E755CB085465DE55DD3940050036B
:1005FD00020A1C855C82855B83E0640B6003020A42
:10060D0017A3E0FFB40A0AE55DB40205D22A020A77
:10061D001CEF6401701E120A5EA3E0640A7015E5FA
:10062D005D6405700F120A5E120A94120A4D1231A2
:10063D0040020A1C120A5EE0B40111120A5EA3E028
:10064D00B40109120C4D121737020A1C120A5EE092
:10065D006401701E120A5EA3E064027015E55D640C
:10066D0005700F120A5E120A94120A4D12619D0254
:10067D000A1C120A5EE06401701D120A5EA3E0649A
:10068D00037014E55DB4050F120A5E120A94FDABFA
:10069D005A123A86020A1C120A5EE0B4011D120AB1
:1006AD005EA3E0B40415E55DD39405400EAB5AADE1
:1006BD005CAC5BAF5D12300C020A1C120A5EE0648A
:1006CD0001701D120A5EA3E064057014E55DB405AA
:1006DD000F120A5E120A94FDAB5A125B0E020A1C2F
:1006ED00120A5EE06401701D120A5EA3E0640670DA
:1006FD0014E55DB4050F120A5E120A94FDAB5A1291
:10070D004DD1020A1C120A5EE0B4011D120A5EA34D
:10071D00E0B40715E55DD39405400EAB5AAD5CAC66
:10072D005BAF5D1245D1020A1C120A5EE0640170D6
:10073D001D120A5EA3E064087014E55DB4050F1286
:10074D000A5E120A94FDAB5A1261D7020A1C120AF4
:10075D005EE0B40215120A5EA3E0B40A0DE55DB4C5
:10076D000308AF5A12635E020A1C120A5EE0B4025D
:10077D0016120A5EA3E0B4010EE55DB40E09120C6B
:10078D004F122D96020A1C120A5EE0B40216120ACE
:10079D005EA3E0B4020EE55DB40709120C4F1252D0
:1007AD00ED020A1C120A5EE0B40215120A5EA3E005
:1007BD00B4090DE55DB40308AF5A125447020A1C83
:1007CD00120A5EE064027019120A5EA3E0B4091108
:1007DD00E55DB4040C120A5E120CB112673F020AF9
:1007ED001C120A5EE064037021120A5EA3E0640A23
:1007FD007018E55D64057012120A5E120A94FD12FE
:10080D006D9BAD5A12473C020A1C120A5EE064034E
:10081D007029120A5EA3E064017020E55DD3940592
:10082D004019120A5E120A94FD126D9B855A62AB35
:10083D005DAD5CAC5B123E15020A1C120A5EE064F3
:10084D00037021120A5EA3E064027018E55D640571
:10085D007012120A5E120A94FD126D9BAD5A125F50
:10086D007E020A1C120A5EE0B40315120A5EA3E0B2
:10087D00B4030DE55DB40308AF5A125FFA020A1C0A
:10088D00120A5EE0B40318120A5EA3E0B40410E588
:10089D005DD394034009120C9A1249D1020A1C121D
:1008AD000A5EE0B40315120A5EA3E0B4050DE55D22
:1008BD00B40308AF5A126D89020A1C120A5EE0B425
:1008CD000316120A5EA3E0B4060EE55DB405091227
:1008DD000C4F126879020A1C120A5EE0640370194B
:1008ED00120A5EA3E0B40711E55DB4040C120A5EB2
:1008FD00120CB1126BA8020A1C120A5EE0B40316A8
:10090D00120A5EA3E0B4080EE55DB40409120C4FA3
:10091D0012689E020A1C120A5EE064057014E55D01
:10092D00B4040F120A54A3A3E0FDAB5A121F8D029B
:10093D000A1C120A5EE0B40516120A98B40B10E5F3
:10094D005DD394054009120C9A123399020A1C12B8
:10095D000A5EE064067014E55DB4040F120A54A338
:10096D00A3E0FDAB5A12217F020A1C120A5EE0B40D
:10097D000616120A98B40B10E55DD39405400912C2
:10098D000C9A1226B0020A1C120A5EE06409701A53
:10099D00120A5EA3E0B40A12E55DB4040D120A5EFC
:1009AD00A3A3E0FF125DAB020A1C120A5EE064090C
:1009BD007018120A5EA3E0B40110E55DB4040B12C9
:1009CD000A5E120CB11262BA8045120A5EE0B409D9
:1009DD0017120A5EA3E0B4020FE55DD3940440083C
:1009ED00120C4D1214F08027120A5EE06409701A81
:1009FD00120A5EA3E0B40310E55DB4040B120A5EA7
:100A0D00120CB1125D1980078000AF5A126BC52010
:100A1D002A030205A2C21ED22DAF5A1259D07D60F3
:100A2D007F021266707D327F031266707F03126E35
:0F0A3D00EF125DF37FFF126EAEE47885F6C223F1
:080A4C0022FD126D9BAD5A2240
:081737008E5E8F5F8D608B61F7
:10173F00120C3BFFE55F2404120AA9FD1264338FDC
:10174F006274E22562F562C394005003021938E512
:10175F006294144003021938E5616406701D120A81
:10176F00A5B4010C120AF4120BF47401F00219342F
:10177F00120AF4120BF4E4F0021934E561640E60FE
:10178F0003021856E55F240C120AA9FFB40A14E5E8
:10179F005F240D120AA9B40A0A120AF4120B84E488
:1017AF00F08013E55F240D120AA9FD126C1C120ABA
:1017BF00F4120B84EFF0E55F240A120AA9FFB40AB2
:1017CF0014E55F240B120AA9B40A0A120AF4120BC9
:1017DF00D2E4F08013E55F240B120AA9FD126C1CF2
:1017EF00120AF4120BD2EFF0E55F2409120AA9FFD7
:1017FF00640A6006EFD39409400A120AF4120BA888
:10180F00E4F08010E55F2409120AA9FF120AF4120E
:10181F000BA8EFF0120AA5FFB40B15E55F24061213
:10182F000AA9B40B0B120AF4120B7474FFF08008A0
:10183F00121964120B74EFF0121940120AE9120B0D
:10184F00F47401F0021934E561640A706E120AF43F
:10185F00120B84E4120AF3120BD2E4F0E55F2409B1
:10186F00120AA9FF640A6006EFD39409400A120A0C
:10187F00F4120BA8E4F08010E55F2409120AA9FF07
:10188F00120AF4120BA8EFF0120AA5FFB40B15E51C
:10189F005F2406120AA9B40B0B120AF4120B74740C
:1018AF00FFF08008121964120B74EFF01219401236
:1018BF000AE9120BF47401F0021934E5616409703E
:1018CF0068120AF4120B84E4120AF3120BD2E41218
:1018DF000AF3120BA8E4F0120AA5FFB40B15E55F8B
:1018EF002406120AA9B40B0B120AF4120B7474FF1C
:1018FF00F08013E55F2406120AA9FD126C1C120A70
:10190F00F4120B74EFF0E55F2407120AA9FFE55FED
:10191F002408120AA9FD126C1C120AF4120AE91209
:10192F000BF47401F0D22C8002C22CAF60126E84C3
:10193F0022E55F2407F582E4355EF583E0FFE55F7E
:10194F002408F582E4355EF583E0FD126C1CE56238
:10195F0075F007A422E55F2406F582E4355EF58372
:0C196F00E0FD126C1CE56275F007A4227C
:103140008F5E8D5FE55ED3941D500302324CE55EC9
:103150009432400302324CD22DAF5F1259D07D46DB
:103160007F07126670AF5E1234C174E2255EF55EB1
:10317000120B80E07021120BCCE0701B120BA2E04E
:103180007015120B6EE0700F120C89700A12326506
:103190007D537F02023242123254E55E75F007A47D
:1031A000120BF4E070047D3680027D387F061266D3
:1031B00070123254120B7EE0FFD394014034EF942E
:1031C00013502F7D097F06126670120B7E12325C3F
:1031D0007FF47E01126C387D0E7F031266707D35A0
:1031E0007F061266707D097F06126670120BCC1284
:1031F000325C7FF47E01126C38120BA2E0FF600596
:10320000125A73800A1232657D0F7F031266707D39
:10321000277F02126670120B6EE0FFF46008126CDA
:10322000D81234C180077D187F021266707D377F07
:1032300004126670120C89FF126CD81234C17D051D
:103240007F06126670C22DAF5F0259D0C22CAF5FED
:10325000126E84227FF47E01126C3822E0FF126C21
:0D326000D81234C1227D187F021266702240
:02619D008D5E15
:10619F00EFD3941D402AEF9432502574E22FFFE481
:1061AF00FEEEFD3395E0FCEF75F007A42450F58269
:1061BF00E4340A120B95E4F00EBE07E5D22C8002F0
:0761CF00C22CAF5E126E84CA
:0161D60022A6
:062D96008E5E8F5F8D6070
:102D9C00D22B120C3BFFE55F2404120AC3122EBD8A
:102DAC00C39418501C855F82855E83A3A3A3E0FFA8
:102DBC00E55F2404120AC3FD126D637883A60780B5
:102DCC0006E47883F6C22B120AB2122EBDC3943CD1
:102DDC00500D120AB2FD126D637884A6078006E4CA
:102DEC007884F6C22BE55F2407120AC3FF126E1615
:102DFC008F61E561D394004017E56194085011E5AB
:102E0C005F2407120AC3FF126E167880A60780068D
:102E1C0078807601C22BE55F2408120AC3FFE55FB8
:102E2C002409120AC3122EC6401FE56194205019C2
:102E3C00E55F2408120AC3FFE55F2409120AC3FDEB
:102E4C00126D637888A607800678887601C22BE518
:102E5C005F240A120AC3FFE55F240B120AC3122E69
:102E6C00C6401FE561940D5019E55F240A120AC390
:102E7C00FFE55F240B120AC3FD126D637881A60770
:102E8C00800678817601C22BE55F240C120AC3FF01
:102E9C00E55F240D120AC3FD126D637882A607301C
:102EAC002B071257BCD22C8002C22CAF60126E843E
:102EBC0022FD1264338F61E56122FD1264338F6150
:062ECC00E561D394002231
:0652ED008E5E8F5F8D60F4
:1052F300D22B120C3BFFE55F2404120BC31253584D
:105303009418501C855F82855E83A3A3A3E0FFE509
:105313005F2404120BC3FD126D637883A607800616
:10532300E47883F6C22B120BB2125358943C500DFF
:10533300120BB2FD126D637884A6078006E47884AD
:10534300F6C22B302B071257BCD22C8002C22CAFD3
:0453530060126E84F2
:0B53570022FD1264338F61E561C32268
:106E1600120C1B4008EF6480948A5001227F0022E6
:106D6300AE05126E16EFC454F0FDAF06126E16EFA9
:036D73004DFF22AF
:10635E008F5ED22D1259D07D1E7F081266707D265B
:10636E007F081266707D527F04126670C22B12680F
:10637E0053125C857880E6FF125A7312597AC22D39
:06638E00AF5E1259D0229F
:10673F008D5EEFD3940A4006EFD3940F4003EF70B2
:10674F000E90002BEFF0D22CAF5E126E84D322C2CC
:08675F002CAF5E126E84C32210
:025447008F5E76
:10544900D22D1259D07D207F051266707D2E7F03E3
:105459001266707D527F0412667090002BE0F55F32
:10546900E55FB40B067D5F7F078034E55FB40C060A
:105479007D5E7F068029E55FB40D067D0A7F028087
:105489001EE55FB40E067D327F028013E55FB40F1F
:10549900067D467F028008E55F70077D0A7F03125B
:0954A9006670C22DAF5E1259D0ED
:0154B20022D7
:106BA8008D5E120C1B400EEF6480948650071263B2
:0D6BB800FFD22C8002C22CAF5E126E842230
:026879008D5E32
:10687B00120C22126433120C1B4010EF648094A193
:10688B005009900029EFF0D22C8002C22CAF5E127F
:02689B006E8409
:01689D0022D8
:02689E008D5E0D
:1068A000120C22126433120C1B4010EF648094A16E
:1068B0005009900028EFF0D22C8002C22CAF5E125B
:0268C0006E84E4
:0168C20022B3
:106D7600D3EF648094814008EF64809489500122A7
:036D86007F002269
:106E2600120C1B4008EF648094A15001227F0022BF
:0814F0008E5E8F5F8D608B6141
:1014F800120C3B14F56374FC2561F5616403600FFD
:10150800E56164076009E561640B60030216D2C3F4
:10151800E5636480948050030216D2E56364809486
:101528008840030216D2E4F562120A8B7803C333AB
:10153800CE33CED8F92430F58274003EF583AF62FD
:10154800EF3395E0FE120B2BE4F00562E562B40878
:10155800D8756204E56164037027120AFB12172D1F
:10156800120A897803C333CE33CED8F9120A6678C3
:1015780003C333CE33CED8F92431F5827400021672
:10158800C9E5616407705D120AFB12172D120A89FA
:101598007803C333CE33CED8F9120A667803C3333F
:1015A800CE33CED8F9120ACCA3120A827803C333F9
:1015B800CE33CED8F91216DAC333CE33CED8F924C7
:1015C80033F5827400120AD2E5822406120B5912EE
:1015D8000A847803C333CE33CED8F92434F5827421
:1015E800000216C9E561640B60030216D2120AFBF9
:1015F800A3E0FD126433126E26120A897803C333FE
:10160800CE33CED8F9120A667803C333CE33CED898
:10161800F9120ACCA3120A827803C333CE33CED888
:10162800F91216DAC333CE33CED8F92433F58274DF
:1016380000120AD2E5822406120B59120A84780392
:10164800C333CE33CED8F92434F5827400120AD2CB
:10165800E5822407120B59120A847803C333CE3368
:10166800CED8F92435F58274003EF583EDF0E562B5
:10167800FD3395E0FC120B0EE5822408F582E43573
:1016880083120B0AE5822409120B59E0FD12643318
:10169800126E26120A897803C333CE33CED8F924C2
:1016A80036F5827400120AD2E582240A120B591206
:1016B8000A847803C333CE33CED8F92437F582743D
:1016C800003EF583EDF0D22C8002C22CAF60126E82
:0116D800848D
:1016D900222432F58274003EF583EDF0E562FD3394
:1016E90095E0FCE55F2DF582E55E3CF583E5822416
:1016F90004F582E43583F583E0FFE55F2DF582E5A6
:101709005E3CF583E5822405F582E43583F583E0C3
:10171900FD126433126E26AD07AF63EF3395E0FE19
:0E172900EF780322A3E0FD126433126E262235
:045D19008D5EAC07E8
:105D1D00D3EC648094804035EC64809489502EE4FB
:105D2D00FDECFF3395E0FEEF7803C333CE33CED8D1
:105D3D00F92428F58274003EF583EDFF3395E0FEDE
:105D4D00120B2BE4F00DBD08D8D22C8002C22CAF63
:045D5D005E126E84E0
:015D6100221F
:1062BA008D5E120C1B402FEF648094895028EF14D6
:1062CA00FFE55E24FF922B124FF9D22DAF5E1259D1
:1062DA00D07542017F327E00126C38E54270FCC2F2
:0762EA002DAF5E1259D02216
:0845D1008F5E8C5F8D608B6131
:1045D900856082855F83120B4CE0FD1264338F6224
:1045E900E562D39400500302467FE56294324003AA
:1045F90002467FE55E64067036D22DAF611259D04E
:104609007D527F05126670AF621234C1120C71B40B
:10461900010A120BDC7401F07D388007120BDCE40F
:10462900F07D367F06126670C22DAF610259D0E562
:10463900602406120C75640B703C120C71B40108ED
:10464900120BDC7401F08005120BDCE4F074F9251F
:104659005EF55E75F00412399AAFF0EF7014E560FB
:104669002406FBE4355FFAAD62E4FF1236BCD22CB6
:0D4679008006C22C8002C22CAF61126E843C
:014686002211
:08300C008F5E8C5F8D608B610B
:10301400856082855F83120B4CE0FD1264338F62FE
:10302400E562D394005003023138E56294284003EA
:10303400023138E55E64067037D22DAF611259D083
:103044007D527F05126670AF621234C1120C0FE01C
:10305400B4010A120BE87401F07D388007120BE802
:10306400E4F07D367F06126670C22DAF610259D03E
:10307400E5602406120C13E0640B6003023138127D
:103084000C0FE0B40108120BE87401F08005120B78
:10309400E8E4F0E4FFFEE5602407120C13E5822E59
:1030A400120B59E0B40B04AF0680040EBE08E7EF20
:1030B4007003023138C39408507A120C7EEFF07E0C
:1030C40001EF2401FDE433FCEEC39DEC6480F8744D
:1030D4008098501DE5602406120C13E5822E120B15
:1030E40059E0FD120C7EE5822E120B59EDF00E8094
:1030F400D0E5602408120C13E5822F120B59E0640A
:103104000B602DEF2408FEC3E55E9EF55E75F004AA
:1031140012399AAEF0EE701CE5602407FDE4355FC9
:10312400FC7E00ED2FFBEE3CFAAD627F011236BC53
:0B313400D22C8002C22CAF61126E840E
:01313F00226D
:0836BC008F638D648A658B6643
:1036C400756801E4F567120B3AE0FF64097037127C
:1036D40037A68003120C56D8FB120B361237987893
:1036E40008EF088003120C56D8FB8E69F56AE5686A
:1036F400FD3395E0FC120CB8E0FF120CB8A3E0FD1A
:10370400126D9B023751120B3AE0FF1237A6800369
:10371400120C56D8FB120B361237987804EF088037
:1037240003120C56D8FB120B36A3A3E0FF126EE56E
:10373400EF426AAE69AF6A7804EF088003120C5650
:10374400D8FB120B36A3A3A3E0FF126EE5EF426A87
:10375400E563700FAF67120A8D120C05E564900AD9
:10376400C08012E563B40117AF67120A8D120C050D
:10377400E564900530120B28E569F0A3E56AF0745E
:10378400042568F5680567C3E56764809490500371
:033794000236CA30
:1037970022A3E0FF126EE5EF426AAE69AF6A22121A
:0E37A7006EE57569008F6AAE697804EF08223E
:0A6EE500EFD3940940037F0022223E
:023A86008B5E55
:103A88001264338F61E561D394005003023B68E50B
:103A98006194334003023B68D22DAF5E1259D07D4A
:103AA800527F05126670AF611234C1746F256112BE
:103AB8000BECE060047D3880027D367F061266706C
:103AC8007F2C7E01126C38E561120C80E0F55F7086
:103AD800077D1B7F061266707D577F02126670E5B0
:103AE8005F603B756001AF5F120A8D2401FFE43E01
:103AF800FEAD60ED3395E0FCC3ED9FEE6480F8EC1D
:103B08006480985019120B19E0B40A04E4FD800689
:103B1800120B19E0FDE4FF126670056080C87F2C67
:103B28007E01126C38E561900530120CD9900000C6
:103B3800EEF0A3EFF04E70077D1B7F061266707DD6
:103B48000C7F03126670900000E07002A3E0600929
:103B5800E56114FD7F01122AF8C22DAF5E0259D02B
:073B6800C22CAF5E126E8457
:013B6F002233
:024DD1008B5EF7
:104DD3001264338F5FE55FD394004077E55F9433CC
:104DE3005071D22DAF5E1259D07D527F051266707D
:104DF300AF5F1234C1749F255F120BE0E060047D46
:104E03003880027D367F061266707F2C7E01126C1D
:104E1300387F2C7E01126C38E55F900AC0120CD9E2
:104E2300900000EEF0A3EFF04E70077D1B7F06129B
:104E330066707D0C7F03126670900000E07002A321
:104E4300E06009E55F14FDE4FF122AF8C22DAF5EAE
:0A4E53000259D0C22CAF5E126E842B
:014E5D002232
:0261D7008B5EDD
:1061D900126433AD07EDD394004025ED943350207C
:1061E900E4FC120BFEED900AC0120B28E4F0A3F0B8
:1061F9000CBC10EE749F2D120BE0E4F0D22C80023F
:07620900C22CAF5E126E848F
:01621000226B
:025B0E008B5EAC
:105B1000126433AD07EDD394004036ED9433503129
:105B2000E4FC120BFEED900530120B28E4F0A3F01C
:105B30000CBC10EE746F2D120BECE4F0FCECFF3398
:105B400095E0FEED120B22E4F00CBC08F0D22C80A4
:085B500002C22CAF5E126E844C
:015B5800222A
:042AF8008F628D63F9
:102AFC00E4F564E5627052AF64120A8D25E0FDEED8
:102B0C0033FCAF63120A8D7805C333CE33CED8F9BC
:102B1C00120B8E120CE58003120C5DD8FB120CC547
:102B2C008003120C5DD8FB540FF566AF63120A8D4F
:102B3C007805C333CE33CED8F9120B8E120CF1803C
:102B4C0003120C5DD8FB022BB6E56264017064AF16
:102B5C0064120A8D25E0FDEE33FCAF63120A8D780A
:102B6C0005C333CE33CED8F92450F5827405120B3D
:102B7C0094120CE58003120C5DD8FB120CC580037B
:102B8C00120C5DD8FB540FF566AF63120A8D7805F5
:102B9C00C333CE33CED8F92450F5827405120B947E
:102BAC00120CF18003120C5DD8FB540FF567ED5439
:102BBC000FF568E565700CE5667008E5677004E56F
:102BCC0068607CAD65E4FF126670AD66E4FF12666A
:102BDC0070E56564097045856769AF69FE7804EF37
:102BEC00088003120C56D8FBF569E5684269E56963
:102BFC00B4990B7D09E4FF1266707D098027E569A5
:102C0C0075F00A84F56AFDE4FF126670E56A75F0EA
:102C1C000AA4FFC3E5699FF56AFD8009AD67E4FF6F
:102C2C00126670AD68E4FF1266707FF47E01126C60
:0F2C3C00380564C3E564648094A05003022AFF46
:012C4B002266
:10643300EFD394004015EF940B5010EFC3940A5020
:1064430008EF75F00AA4FE8002E4FEEDD394004049
:106453000EED940B5009EDC3940A5003ED2EFEAFDD
:016463000632
:016464002215
:0649D1008E5E8F5F8B601B
:1049D700756105756240D3ED64809484407CED6415
:1049E7008094A55075ED24FDF563D39404406BE5E1
:1049F7006320E06613F5640562E562AE6170020547
:104A07006114F5828E83E564F07403255FF55FE436
:104A1700355EF55EE4F563E563C395645033855F02
:104A270082855E83E0FFA3E0FD126D9B0562E56270
:104A3700AC617002056114F5828C83EFF0055FE5C8
:104A47005F7002055E055FE55F7002055E056380C6
:104A5700C6D22CAF60126E84D322C22CAF60126E06
:024A670084C306
:014A6900222A
:043E15008C5F8D60D1
:103E1900120C1B5003023EEDEF648094954003029F
:103E29003EEDEB648094875003023EEDEB64809491
:103E3900E44003023EED120A8D7805C333CE33CE3A
:103E4900D8F9120D1FF5638F64EB24FBF565D39444
:103E5900025003023EEDE56575F00384E5F0600369
:103E6900023EEDE56575F00384F567C3941050745F
:103E7900120CD27002056314F5828E83E567F07423
:103E890005120D29E4F565E565C395675052120DD4
:103E990033E0F566B40A10120CD27002056314F50A
:103EA900828E83E4F0800F120CD27002056314F540
:103EB900828E83E566F0120D33A3E0FF120D33A362
:103EC900A3E0FD126D9B8F66120CD270020563147C
:103ED900F5828E83E566F07403120D29056580A7C6
:0B3EE900D22C8002C22CAF62126E844B
:013EF40022AB
:0826B0008E5E8F5F8D608B616F
:1026B800C22B120D3A600302274D1228285003023C
:1026C8002748E5649408E56394075074C3E560649B
:1026D80080948A506B120C44A3E0F562B401069012
:1026E800052002279DE562B4020690052202279D77
:1026F800E562B4030690052402279DE562B404064A
:1027080090052602279DE562B40506900528022754
:102718009DE562B4060690052A02279DE562B40786
:102728000690052C02279DE562B4080590052E80C9
:1027380064E562B40905900530805AD22B02281945
:10274800D22B022819120C44E064017052AD60AF1C
:102758005FAE5E1228285003022819E5649408E544
:102768006394074003022819C3E5606480948A4093
:1027780003022819120C44A3E0F562B40A05900577
:10278800328012E562B401059005348008E562B430
:102798000209900536E563F0A3806FD22B80721290
:1027A8000C44E06402706AAD60AF5FAE5E125B59C4
:1027B8007563008F64C3E5649463E56394005051C6
:1027C800C3E560648094885048120C44A3E0F56225
:1027D800B40107900538EFF08037E562B402059040
:1027E80005398026E562B4030590053A801CE56248
:1027F800B4040590053B8012E562B4050590053CDC
:102808008008E562B4060890053DE564F08002D2D0
:0F2818002B302B04C22C8002D22CAF61126E84A5
:10282700221248908E638F64D3E564943BE56394EA
:0228370000227D
:064890008E658F66A9058C
:104896007D057C00120D09E0C3940A4005120D093E
:1048A600E4F00DBD00010CED640A4C70E7B9060793
:1048B600120B61FF7E0022E964077010120B61750E
:1048C600F00AA4ACF0FDE5662406801BE9640870D6
:1048D60021120B6175F064A4ACF0FDE566240612A6
:1048E6000B65120C642407120B652DFDE43CAF0525
:1048F600FE22E964097033120B61FF7E007C037DA2
:10490600E81239BCAC06AD07E5662406120B6575E0
:10491600F064120C672407120B65120C642408124B
:0D4926000B652DFDE43CFEAF0522E4FEFF15
:014933002261
:065B59008E658F66A905B0
:105B5F007F057E00120D14E0C3940A4005120D1448
:105B6F00E4F00FBF00010EEF64084E70E7E9640721
:105B7F007020E5662405F582E43565F583E075F060
:105B8F000AA4FFE5662406F582E43565F583E02F68
:045B9F00FF227F0062
:015BA30022DF
:083399008E5E8F5F8D608B6179
:1033A100C22BD3E560648094845003023447E56006
:1033B1006480948D4003023447120D3A6003023455
:1033C10047120C3B123A6033E70133F20233FD033B
:1033D100340704341105341B06342507342F08340F
:1033E100390900003443756201756300D22B023440
:1033F1007E756201756308D22B02347E7562017598
:103401006310D22B8077756201756318D22B806DA2
:10341100756201756320D22B806375620175632823
:10342100D22B8059756201756330D22B804F756242
:1034310001756338D22B8045756201756340D22BCB
:10344100803BC22B8037D3E56064809484402EE5B5
:10345100606480948D5026855F82855E83A3A3E09E
:10346100B4011A855F82855E83A3A3A3E024F6706D
:103471000A756201756358D22B8002C22B302B383A
:10348100E4FF120CA3E4F00FBF08F7E56024FB850D
:103491006382856283F07F01E55F2404F582E43570
:1034A1005EF583E5822F120B59E0FE120CA3EEF0BC
:0F34B1000FBF08E4D22C8002C22CAF61126E84D0
:0134C00022E9
:04473C008F5E8D5FA0
:10474000E55ED3940050030247DFE55E9415400315
:104750000247DFD22DAF5F1259D07D5F7F05126611
:1047600070AD5EE4FF1266707D527F041266707F4A
:10477000F47E01126C3875F020E55E900280123AEA
:1047800054AF828583628F63E0F560603DD394000F
:104790004046E56094105040E56025E0F5607561A5
:1047A00001E5602401FFE433FEC3E5619FEE648010
:1047B000F87480985022120CFDE0FF120CFDA3E06B
:1047C000FD1265280561056180D77D1B7F06126695
:1047D000707D5F7F05126670C22DAF5F0259D0C237
:0647E0002CAF5F126E8495
:0147E60022B0
:10217F008F5E8D5F8B60E55E640A7074E55FC3945C
:10218F000A40030222EC122322E4FDFF126670AD17
:10219F005F1222FBE55F123A6021C70121CD0221B8
:1021AF00D30321D90421DF0521E50621EB0721F116
:1021BF000821F709000021FC900520022246900516
:1021CF00220222469005240222469005260222462C
:1021DF0090052802224690052A02224690052C02DD
:1021EF00224690052E022246900530804A0222E5B3
:1021FF00E55E64017052E55FD394004006E55F949D
:10220F00034006E55F640A703C122322E55FB40ABF
:10221F000A7D0A1222FB900532801CE55FB4010A89
:10222F007D0B122308900534800DE55FB402137DFA
:10223F000C122308900536E0FEA3E0FF126497020C
:10224F0022F30222E50222ECE55E64026003022221
:10225F00F3E55FD3940050030222ECE55F9407503F
:10226F007CD22DAF601259D07D277F081266707D0A
:10227F0006E4FF1266707D14E4FF126670E55F24BA
:10228F00FE601A14602114602814602F1460362425
:10229F000570437D0112231590053880307D0212A1
:1022AF00231590053980267D0312233890053A8037
:1022BF001C7D0412233890053B80127D05122345A7
:1022CF0090053C80087D0612234590053DE0FF7E7A
:1022DF00001264C8800EAF60126BC58007C22CAFAE
:1022EF0060126E84C22DAF601259D022E4FF1266C5
:1022FF00707D527F0412667022E4FF1266707D5269
:10230F007F0412667022E4FF1266707D527F041202
:10231F00667022D22DAF601259D07D277F081266CA
:10232F00707D06E4FF12667022E4FF1266707D5224
:10233F007F0412667022E4FF1266707D527F0412D2
:03234F0066702293
:044B02008E638F64CB
:104B06000564E5647002056314F5828E83E0F5663C
:104B1600607AC3940850757F2C7E01126C38E4F5D8
:104B260065E565C395665064856482856383E01296
:104B36003A604B73004B510A4B550B4B5B0C4B6168
:104B46000D4B670E4B6D0F00004B79E4FD802D7DFC
:104B56005F7F0780287D5E7F0680227D0A7F028038
:104B66001C7D327F0280167D467F0280107D0A7F83
:104B760003800A856482856383E0FDE4FF12667024
:0C4B86000564E564700205630565809518
:014B92002200
:061F8D008F5E8D5F8B608A
:101F9300C22BE55E640A6003022081E55F123A60AA
:101FA3001FC2011FD5021FE8031FFB04200E0520DB
:101FB3002406203A072050082065090000207D12DE
:101FC30020B67D01122104756101756200D22B02D6
:101FD300209D1220B67D02122104756101756208ED
:101FE300D22B02209D1220D27D0312211175610193
:101FF300756210D22B02209D1220D27D0412211172
:10200300756101756218D22B02209D1220EE1221F8
:10201300647D05122134756101756220D22B022083
:102023009D1220EE1221647D061221347561017523
:102033006228D22B02209D12211E1221787D0712C5
:102043002141756101756230D22B02209D12211E40
:102053001221787D08122141756101756238D22BF6
:10206300803812214EE4FDFF1266707D0912216B48
:10207300756101756240D22B8020C22B801CE55E06
:1020830064017016E55F24F6701012214E7D0A126A
:10209300216B756101756258D22B302B09AF62AE8B
:1020A30061124B028005AF60126BC5C22DAF601287
:0220B30059D002
:1020B50022D22DAF601259D07D577F021266707DF6
:1020C50005E4FF126670E4FDFF12667022D22DAFA3
:1020D500601259D07D577F021266707D05E4FF12AC
:1020E5006670E4FDFF12667022D22DAF601259D0E2
:1020F5007D577F021266707D05E4FF12667022E44B
:10210500FF1266707D527F0412667022E4FF12662C
:10211500707D527F0412667022D22DAF601259D0A5
:102125007D577F021266707D05E4FF12667022E41A
:10213500FF1266707D527F0412667022E4FF1266FC
:10214500707D527F0412667022D22DAF601259D075
:102155007D577F021266707D05E4FF12667022E4EA
:10216500FDFF12667022E4FF1266707D527F041235
:0A217500667022E4FDFF126670227E
:1034C1008F72E572D3945940107D5A1235A824A603
:1034D100FD70030235A70235A2E572D3944F401661
:1034E100E572945A50107D501235A824B0FD700336
:1034F1000235A70235A2E572D394454016E57294D0
:103501005050107D461235B024BAFD70030235A724
:103511000235A2E572D3943B4012E5729446500CF9
:103521007D3C1235B024C4FD607C8075E572D39476
:10353100314012E572943C500C7D321235B824CEE4
:10354100FD6063805CE572D394274012E57294328A
:10355100500C7D281235B824D8FD604A8043E572AD
:10356100D3941D4016E572942850107D1EE4FF127D
:103571006670E57224E2FD602D8026E572D3941316
:103581004016E572941E50107D14E4FF126670E53A
:103591007224ECFD60108009E572C394145007ADEC
:1035A10072E4FF12667022E4FF126670E57222E493
:0F35B100FF126670E57222E4FF126670E5722267
:1059D0008F6AE56A700C302D097F01126F027FC05B
:1059E000801FE56A700C202D097F01126EEF7FC0C9
:1059F0008026E56AB40112302D0F7F02126F027FFC
:105A000030120016C22F02697AE56AB40114202D03
:105A1000117F02126EEF7F30126EAE7FC87E0012D1
:035A20006C3822BD
:106956008F69D22D1259D07D607F021266707D320A
:106966007F061266707D1E7F05126670C22DAF69A6
:046976001259D022C0
:106BC5008F69D22D1259D07D607F021266707D309B
:0D6BD5007F03126670C22DAF691259D022E5
:0E6E84008F68302C03026956AF68126BC5226E
:105DAB00EF24FE60101460162402701C7F01126F2A
:105DBB00027F8080107F02126F027F2080077F039B
:105DCB00126F027FA01200167FF47E01126C3875E1
:105DDB004204E54270FC7F647E00126C387F031234
:085DEB006EEF7FA0126EAE22E4
:1064C8008E618F627C007D0A1239CEAD07E4FF121F
:1064D80066707D5B7F06126670AE61AF627C007D80
:1064E8000A1239CEE4FF1266707D4A7F0702667091
:046497008E618F6221
:10649B007C007D3C1239CE1234C17D057F0612661D
:1064AB0070AE61AF627C007D3C1239CEED4C600C5E
:0C64BB00AF051234C17D4A7F07126670E5
:0164C70022B2
:025F7E008D5E36
:105F8000120C1B402FEF648094955028120A8D78D4
:105F900005C333CE33CED8F9120D1FFEE4FD0FEF4B
:105FA000AA0670010E14F5828A83E4F00DBD20EE7E
:0B5FB000D22C8002C22CAF5E126E8467
:015FBB0022C3
:105FFA008F5E900540E0D394024015D22D1259D0FD
:10600A007542037F327E00126C38E54270FC8015BF
:10601A00D22DAF5E1259D07D1B7F061266707D0CA1
:0D602A007F03126670C22DAF5E1259D022A6
:106D89007E10900540E4F0A3DEFC7E10D22C126E3A
:016D99008475
:016D9A0022D6
:106D9B00BF0A02E4FFBD0A02E4FDEF75F00AA42D61
:026DAB00FF22C5
:106C1C00EFD394094002E4FFEDD394094002E4FD64
:0C6C2C007804EF08800123D8FD4DFF2202
:10409C0007010203040506070707060504030201CE
:1040AC0003010A0A030307050303020503020A0AB4
:1040BC0004050A0A0104050A0A0A04050A0A02038D
:1040CC00070A0A03040A0A04024B00020032072EF4
:1040DC0003024B0002003202055F000302055F0081
:1040EC000402055F000502055F000604072E082682
:1040FC000640033204072E08260640025304081E0D
:10410C0008260452010008024B00020032072E0858
:10411C001E08260452010003072B0235063603073E
:10412C002B0235063803072B0235072603072B0213
:10413C0035025302055F000F02055F001002055F98
:10414C00001102055F001202055F001302055F00FB
:0A415C0014080C0A1D020500241BC4
:105274007461F0A37420F0A37452F0A37401F0A33A
:1052840022A3F0A37461F0A37440F022F0A374038A
:10529400F0E4A3F0A37410F0A37403F0E4A3F0A368
:1052A400227461F0A37441F0A3227461F0A3F0A30B
:1052B4007430F0A3227496F0A37432F0A37495F0C2
:1052C400A3741EF0A322F0A37461F0A314F0A374DA
:1052D40070F0A3E4F022A3F0A37452F0A3223CF5EF
:0952E40083E0FEEF3395E0FC22AB
:10003E007E407F9C7C017D507B081260EC7E407F71
:10004E00A47C017D587B081260EC7E407FAC7C0165
:10005E007D007B041260EC7E407FB87C017D087BC6
:10006E00041260EC7E407FB47C017D107B04126034
:10007E00EC7E407FB07C017D187B041260EC7E40EC
:10008E007FC17C017D207B051260EC7E407FBC7CB5
:10009E00017D287B051260EC7E407FC67C017D30A1
:1000AE007B051260EC7E407FCB7C017D387B041299
:1000BE0060EC7E407FCF7C017D407B041260EC7E45
:1000CE00407FD37C027DA07B091260EC7E407FDCFA
:1000DE007C027DC07B071260EC7E407FE37C027D5C
:1000EE00E07B051260EC7E407FE87C037D007B05A3
:1000FE001260EC7E407FED7C037D207B051260EC70
:10010E007E407FF27C037D407B051260EC7E407F5B
:10011E00F77C037D607B091260EC7E417F007C03DF
:10012E007D807B091260EC7E417F097C037DA07B84
:10013E00091260EC7E417F127C037DC07B11126040
:10014E00EC7E417F237C037DE07B071260EC7E41D9
:10015E007F2A7C047D007B071260EC7E417F317C20
:10016E00047D207B071260EC7E417F387C047D404D
:10017E007B071260EC7E417F3F7C047D607B051225
:10018E0060EC7E417F447C047D807B051260EC7EBA
:10019E00417F497C047DA07B051260EC7E417F4E41
:1001AE007C047DC07B051260EC7E417F537C047D18
:1001BE00E07B051260EC7E417F587C057D007B055F
:1001CE001260EC7E417F5D7C057D407B091260EC08
:1001DE009000297417F07F031263FF9000287419A2
:1001EE00F090002074B1F09000217491F0900022F4
:1001FE007403F0900023747FF090002404F09000BC
:10020E00257403F0E4900026F0900027F090003063
:10021E0074091252907415F0A37403F0A37415129E
:10022E0052907409F0A37403F0E4FFEFFD3395E0F0
:10023E00FC74302DF58274001252E274102DF5828A
:10024E0074003CF583EEF00FBF08E0E4FFEFFD33E2
:10025E0095E0FC74382DF58274001252E274182D5C
:10026E00F58274003CF583EEF00FBF08E090052098
:10027E00E4F0A374B4F0900522E4F0A374B4F0900B
:10028E0005247401F0A374E0F0900526E4F0A37445
:10029E0078F09005287402F0A37458F090052AE4C3
:1002AE00F0A3743CF090052C7402F0A37458F07413
:1002BE000790052EF0A3F0900530F0A3F0900532D4
:1002CE00F0A3F0900534F0A3F0900536E4F0A3749B
:1002DE003CF0900538740AF09005397428F09005BA
:1002EE003A7405F090053B740AF090053CF09005C9
:1002FE003D7428F09000A47401F0900B607415F01A
:10030E00A37411F09000A57401F0900B807415F099
:10031E00A37410F09000A67401F0900BA07415F069
:10032E00A37421F09000A77401F0900BC07415F027
:10033E00A37420F09000A87401F0900BE07415F0F7
:10034E00A37431F09000A97401F0900C007415F0B4
:10035E00A37430F09000AA7401F0900C207415F084
:10036E00A37441F09000AB7401F0900C407415F042
:10037E00A37440F09000AC7401F0900C60745312B2
:10038E00527E743612527E7438F0A3E4F0A3745386
:10039E00F0A3E4F09000AD04F0900C807453125270
:1003AE007E7434F0A37421F0A37453F0A3E4F090A0
:1003BE0000AF04F0900CC012527C7430F074031233
:1003CE0052DAE4F09000B004F0900CE012527C741B
:1003DE0030F074041252DAE4F09000B104F0900D93
:1003EE0000125274743212527E7452F0A37420F0C2
:1003FE009000B27401F0900D201252747432F0A37A
:10040E0074021252DB7420F09000B37401F0900D60
:10041E0040745312527E7433F0A3E4F09000B4048F
:10042E00F0900D601252A57430F074021252859045
:10043E0000B57401F0900D801252A57430F0740561
:10044E001252859000B67401F0900DA01252A57450
:10045E0030F0A374061252869000B77401F0900D1E
:10046E00C01252A51252B97498F0A3744B12528650
:10047E009000B87401F0900DE01252A51252B974AA
:10048E0093F0A374181252869000B97401F0900E76
:10049E00001252A57430F0A37413125286A3747016
:1004AE00F0A37402F09000BA14F0900E201252AE27
:1004BE007412F0A3747012527E7461F0A314F09053
:1004CE0000BB7401F0900E401252AE74111252CA5B
:1004DE009000BC04F07461900E601252B07414124D
:1004EE0052CA9000D104F09011001252A57492F0ED
:1004FE00A3744BF0A37490F0A37402F0A37490F065
:10050E00A37432F07499A3F0A3F0A3746012527E18
:10051E00749112527E7491F0A3E412528690000FE1
:10052E007401F0125DF37F01126F027F401200160C
:10053E007D2F7F071266707D0C7F031266707D32F1
:0C054E007F061266707D1E7F051266702D
:01055A00227E
:0A60EC008E5A8F5B8C5C8D5D8B5E1D
:1060F600E4F9C3E55E6480F8E96480985022E9FF1C
:106106003395E0FEE55B2FF582E55A3EF583E49391
:10611600FDE55D2FF582E55C3EF583EDF00980D265
:016126002256
:10558200AF6AEF3395E0FEE56975F008A42428F5CB
:1055920082E43400F583E5822FF582E5833EF583CC
:1055A200E0FFE56AFD3395E0FC22AB66AD65AF64D2
:1055B200223EF583E0FD74B82FF582741D3EF5831B
:1055C200EDF0056AE56A22EF3395E0FEEF25E0FF94
:1055D200EE33FE22A2E0CE13CE13223CF583EFF08F
:0555E200056AE56A22E4
:045BA4008C5B8D5C2D
:105BA800EF6043D201D202D20CE4F55D855C8285B8
:105BB8005B83E0FEA3E04E6027AF5D1255C9E55C4C
:105BC8002FF582E55B3EF583E0FEA3E0FF12451961
:105BD800922920290B055DC3E55D6480949040CC33
:065BE800C201C202C20C62
:015BEE002294
:045BEF008C608D61D8
:105BF300EF6043D201D202D20CE4F5628561828563
:105C03006083E0FEA3E04E6027AF621255C9E561F1
:105C13002FF582E5603EF583E0FEA3E0FF12451910
:105C2300922D202D0B0562C3E5626480949040CCD5
:065C3300C201C202C20C16
:015C39002248
:04451900AD07AC0638
:10451D00C22E780CEF0880031255D6D8FB540FF538
:10452D00637808AF05AE04EF0880031255D6D8FBAB
:10453D00540FF5647804AF05AE04EF0880031255EF
:10454D00D6D8FB540FF565ED540FF566E563607134
:10455D00B401081255AC123C538066E563B40208F1
:10456D001255AC126B308059E563B403081255AC8B
:10457D001238AC804CE563B404081255AC126AD104
:10458D00803FE563B405081255AC1225028032E573
:10459D0063B406081255AC1212828025E563B40788
:1045AD00081255AC125AC28018E563B408081255AA
:1045BD00AC125761800BE563B409061255AC126855
:0345CD00C3A22E58
:0145D00022C8
:103C53008F678D688B69E567B40113900020E0FFDF
:103C63001258CA900020EFF0FD7F20023D10E56757
:103C7300B40211900021123D16900021EFF0FD7F58
:103C830021023D10E567B40311900022123D169006
:103C93000022EFF0FD7F22023D10E567B40410908F
:103CA3000023123D20900023EFF0FD7F23805EE58B
:103CB30067B40516900024123D20900024EFF0FD18
:103CC3007F247E001263940264F8E567B4061090C3
:103CD3000025123D2A900025EFF0FD7F25802EE57B
:103CE30067B40710900026123D2A900026EFF0FDDE
:103CF3007F268019E567B40819900027E0FFAB69B8
:103D0300AD681258CA900027EFF0FD7F277E00129E
:103D1300639422E0FFAB69AD681258CA22E0FFAB9F
:103D230069AD681258CA22E0FFAB69AD681258CA80
:013D3300226D
:1058CA00D22FAC07BD01047E018033BD02047E02E3
:1058DA00802CBD03047E048025BD04047E08801E3E
:1058EA00BD05047E108017BD06047E208010BD070A
:1058FA00047E408009BD08047E808002C22FBB015D
:10590A0005EE4204800BEB7006EEF452048002C2EC
:07591A002F302F03AF042220
:015921002263
:026B30008B6771
:106B3200C22FEF7016ED7013E5677003025C85E5F6
:0B6B420067B401077880E6FF125A7369
:016B4D002225
:0638AC008F678D688B6937
:1038B200E5677007123992E4FD801AE567B40107E3
:1038C2001239927D01800EE567B4020CAD69AF68D2
:1038D200126E927D02024F71E567B40306124D42E9
:1038E200C21E22E567B40415AD69AF681264338F56
:1038F20043754205E542700302399180F7E567643A
:10390200067017E5687013F56A12558274102DF56A
:103912008274001255DDB408F022E567640770175F
:10392200E5687013F56A12558274182DF5827400D9
:103932001255DDB408F022E56764087027E5687067
:1039420023E569701FF56AAF6AEF3395E0FE7410E4
:103952002FF58274001255B3B408EC754201E542AA
:10396200602D80FAE56764097025E5687021E569D4
:10397200701DF56AAF6AEF3395E0FE74182FF58279
:0F39820074001255B3B408EC754201E54270FCB5
:0939910022AD69AF68126E9222AA
:106AD1008F67AE03AF05E567D394004012E5679475
:106AE10007500CAD06126E92AD07AF671266C42255
:102502008F678D688B69E5677018E5687014E569F7
:1025120070057F01126EAEE569640160030226AFA9
:102522008043E567701CE568B40117E56970057FB3
:1025320004126EAEE569640160030226AF7F0402F5
:1025420026ACE5677029E56864027023E5697005C9
:102552007F05126EAEE569640160030226AF90004A
:102562000FE0B403057F010226AC7F050226ACE52D
:1025720067B4011BE5687017E56970057F02126E8A
:10258200AEE569640160030226AF7F020226ACE574
:1025920067B4011CE568B40117E56970057F08128C
:1025A2006EAEE569640160030226AF7F080226ACC5
:1025B200E56764017029E56864027023E5697005C6
:1025C2007F0A126EAEE569640160030226AF9000D5
:1025D2000FE0B403057F020226AC7F0A0226ACE5B7
:1025E20067B4021BE5687017E56970057F40126EDB
:1025F200AEE569640160030226AF7F400226ACE5C6
:1026020067B4021CE568B40117E56970057F101212
:102612006EAEE569640160030226AF7F100226AC4C
:10262200E56764027024E5686402701EE56970055E
:102632007F50126EAEE5696401707290000FE0B4D3
:1026420003047F4080647F508060E567B40317E530
:10265200687013E56970057F80126EAEE5696401EA
:10266200704B7F808044E567B40318E568B40113BA
:10267200E56970057F20126EAEE5696401702E7FF8
:10268200208027E56764037024E5686402701EE514
:102692006970057FA0126EAEE569B4011090000F5B
:0E26A200E0B403047F8080027FA012001622A5
:101282008F678D688B69E5677017AD69AF68126EFD
:10129200928E348F35D3E5359400E534940050F5C1
:1012A20022E567B4011BE568B40116E5697007C25F
:1012B200307F01122ED2E569640160030214EF80CF
:1012C20058E5676401702BE56864027025E5697072
:1012D20007C2307F02122ED2E56964016003021454
:1012E200EF90000FE0640370030214EFD2307F022C
:1012F2008031E5676401702EE56864037028E56952
:101302007007C2307F03122ED2E5696401600302C6
:1013120014EF90000FE0B40306D2307F018004D2B4
:10132200307F03022ED2E5676401702DE568640404
:101332007027E569700CC2307F01122ED27F4012F5
:101342006EAEE569640160030214EFD2307F0112D0
:101352002ED27F40120016807CE5676401703AE568
:101362006864057034E569700CC2307F02122ED2B7
:101372007F10126EAEE569640160030214EF900003
:101382000FE0640370030214EFD2307F02122ED2F8
:101392007F10120016D22F803EE5676401703BE594
:1013A2006864067035E569700CC2307F03122ED274
:1013B2007F50126EAEE569640160030214EFD23011
:1013C2007F03122ED290000FE0B403047F4080020C
:1013D2007F50120016C22F02697AE56764027029F3
:1013E200E56864017023E56970057F100214D6E593
:1013F20069B401057F100214E0E56964026003022A
:1014020014EFD22F7F010214ECE56764027029E524
:101412006864027023E56970057F200214D6E569CD
:10142200B401057F200214E0E5696402600302143E
:10143200EFD22F7F020214ECE56764027029E5689F
:1014420064037023E56970057F400214D6E569B430
:1014520001057F400214E0E569640260030214EFB3
:10146200D22F7F030214ECE56764027023E56864FF
:1014720004701DE56970047F808059E569B4010438
:101482007F80805AE56964027063D22F7F04805A9C
:10149200E56764027023E5686405701DE569700400
:1014A2007F048030E569B401047F048031E569641A
:1014B20002703AD22F7F058031E5676402702EE513
:1014C20068640670287D017F07124EE9401FE569B6
:1014D20070057F08026EEFE569B401057F08026FAF
:0E14E20002E569B40207D22F7F0612299A2272
:025AC2008B67F0
:105AC400EF7037ED7034E567700690000F048020A6
:105AD400E567B4010A90000F7402F0D22F801BE531
:105AE40067B40216C21E7FFF126EAE90000F7403DD
:105AF400F0C2307F02122ED2D22F302F0C90000F22
:095B0400E0FD7F0F7E00126394A6
:015B0D002275
:105761008F678D688B69E567700C1257A5749F2F41
:10577100F58274008019E567B4010C1257A5749F76
:105781002FF58274008016E567B402091257AD3E09
:10579100F583E4F022E567B403091257AD3EF583C2
:1057A1007401F022AD69AF68126E9222AD69AF68E3
:0B57B100126E92746F2FF582740022BC
:0268C3008F67DD
:1068C500AF057804EF08800123D8FD4BF568E5672F
:1068D500B40908E568B499030253D7AD68AF6712E8
:0268E500652824
:0168E700228E
:0D6E9200EF75F00AA47C002DFFEC35F0FE3A
:016E9F0022D0
:0466C4008F688D69E5
:1066C800C3E569648094E4501BE4F56AC3E5696432
:1066D80080F8E56A648098500BC22FAF6812299A37
:0466E800056A80E8D7
:0166EC00228B
:0D6EA000C296007F0512682D126465D2961F
:016EAD0022C2
:106D3700126EA0EF20E0F9C296007F0612682DC2FE
:066D4700B60000D2962206
:106D4D00126EA0EF20E0F9C296007F0412682DC2EA
:066D5D00B60000D29622F0
:045FBC008E608F6103
:105FC000AE04AF058E638F64C296007F0312682D06
:105FD000E560FF12682DAF6112682DE4F56212646E
:105FE00065E5642562F582E43563F583EFF00562CB
:095FF000E562C3942040E7D2965B
:015FF9002285
:085C3A008E658F668C678D6892
:105C4200126EA0EF20E0F985656A85666BC2960048
:105C52007F0212682DE567FF12682DAF6812682D6A
:105C6200E4F569E56B2569F582E4356AF583E0FFC1
:105C720012682D0569E569C3942040E7C2B60000A9
:025C8200D296B8
:015C840022FD
:0A551C008E5A8F5B8C5C8D5D8B5EF8
:10552600C2AF126D37126EA0EF20E0F9855C608580
:105536005D61C296007F0212682DE55AFF12682D42
:10554600AF5B12682DE4F55FAF5EEF3395E0FEC307
:10555600E55F9FEE6480F87480985014E561255FDE
:10556600F582E43560F583E0FF12682D055F80D88B
:0B557600C2B60000D296126D4DD2AFFD
:015581002207
:106394008E718F728D73C2AF126D37126EA0EF20A3
:1063A400E0F9C296007F0212682DE571FF12682D94
:1063B400AF7212682DAF7312682DC2B60000D29668
:0663C400126D4DD2AF2264
:10607400C2AFE4F55BF55CF55DF55EF55FF55AAE30
:106084005EAF5FAC5BAD5C125FBC7420255CF55CFD
:10609400E4355BF55B7420255FF55FE4355EF55E02
:0B60A400055AE55AC3948940D6D2AFDC
:0160AF0022CE
:105DF300C2AF756200756300756400E4F560F56118
:105E0300F55F126D37AE63AF64AC60AD61125C3A9F
:105E130074202561F561E43560F56074202564F52F
:105E230064E43563F563055FE55FC3948940D3128A
:045E33006D4DD2AF30
:015E37002248
:105649000500050105030507050F051F051E051CB6
:10565900051805100201040E040A03060101040BD2
:105669000304040F020304010302040D02000202F1
:1056790003000409040403050307010003030407E5
:10568900030104060402040C05160515000006159D
:0E569900062A060C06380633061E06120617F1
:104CB3002430F58274003EF583EDFF3395E0FEE585
:104CC300822FF582E5833EF583E0FFEDFB3395E02C
:104CD300FA22AF4112682DC293126EF9D293D2AF6A
:104CE300223EF583E0FC74B82FF582741D3EF583F4
:104CF300ECF00D221528E528D394002225E0244961
:104D0300F582E43456F583E49322E4F57CD20EC2B3
:104D130027C21DC21A227FA0126EAEE4F542C21E44
:104D230022126EF9D2B67801EF0822122C4CD2CAA5
:0F4D3300D20ED22722ECFF3395E0FEEF78032259
:10416600200E2F900540E004F577D36480948150AB
:1041760003024226D3E5776480948F400375770F58
:10418600900029E0FF122C4C90002AE0F576124DA3
:104196000D22301A58302712124CF74003024226DD
:1041A600C2CAC227D21D85762822301D0A124CF7B4
:1041B600506EC227C21D22AF7A157AEF700BC21A53
:1041C600E57625E0F528D21D22E57B30E0058576EB
:1041D600288008E57675F003A4F528AF7B7801EF13
:1041E60008800103D8FDF57BD227D2CA22D57708ED
:1041F600C20EE4F542C21E22057C7440257CF5827F
:10420600E43405F583E0124CFF540FF57A740193FC
:10421600F57B700AD21DE57625E025E0F528D21A51
:014226002275
:10510200200E12900029E0FF122C4C90002AE0F5AC
:1051120078124D0D22301A5130270F124CF7505D84
:10512200C2CAC227D21D85782822301D0A124CF726
:10513200504BC227C21D22AF7A157AEF7007C21AEE
:10514200C20EF54222E57B30E0058578288008E52D
:105152007875F003A4F528AF7B7801EF088001038E
:10516200D8FDF57BD227D2CA22E543124CFFFA744E
:0D5172000193FBEA540FF57AEBF57BD21A9E
:01517F00220D
:10646500E4F575D297F574C2B6126EF9AF75780179
:10647500EF08800123D8FDF57530970343750112A8
:106485006EF9D2B60574C3E5746480948840D8AFBC
:016495007591
:0164960022E3
:096EF9000000000000000000226E
:10664400C2B7E4FEC2B6126EF9EF30E704D2B580E9
:1066540002C2B5124D24800123D8FDFF126EF90E3B
:0B666400BE08E1C2B6D2B7D2B6D2B574
:01666F002208
:0D001600C2AFEF4227AF27126644D2AF22DF
:0E6EAE00C2AFEFF45227AF27126644D2AF22D4
:10682D00E4FEC2B6126EF9EF30E704D2B58002C2B3
:10683D00B5124D24800123D8FDFF126EF90EBE084E
:05684D00E1D2B6D2B556
:016852002223
:096F0200C2AFEF4241124CD5224E
:0A6EEF00C2AFEFF45241124CD5225D
:102C4C00EF123A602CB4012CBB022CC2032CC90429
:102C5C002CD0052CD7062CDE072CE5082CEC092CE7
:102C6C00F30A2CFA0B2D010C2D080D2D0F0E2D1621
:102C7C000F2D1D102D24112D2B122D32132D391427
:102C8C002D40152D47162D4E172D55182D5C192D31
:102C9C00631A2D6A1B2D711C2D731D2D7A1E2D810F
:102CAC001F2D882000002D7175CB8E75CAC622751C
:102CBC00CB9575CA772275CB9B75CA692275CBA04B
:102CCC0075CABA2275CBA675CA332275CBAB75CA39
:102CDC00632275CBB075CA022275CBB475CAA32218
:102CEC0075CBB875CAFA2275CBBC75CAD82275CB10
:102CFC00C075CAA82275CBC475CA362275CBC775E8
:102D0C00CA862275CBCA75CABC2275CBCD75CAB41E
:102D1C002275CBD075CA762275CBD375CA30227585
:102D2C00CBD575CAB22275CBD875CA132275CBDA3E
:102D3C0075CA522275CBDC75CA7D2275CBDD75CA7E
:102D4C006E2275CBE075CA542275CBE275CA1B2274
:102D5C0075CBE375CAC32275CBE575CA5E2275CBFC
:102D6C00E675CADA22801C75CBE875CA902275CB41
:102D7C00EA75CAD92275CBEC75CA092275CBED75EB
:0A2D8C00CA292275CBE875CA41225E
:10002600C3EF648094A15008EF25E025E0F528226F
:04003600E4F52822A3
:0237B5008F5A29
:1037B700900118E0FFE55A7006E545D39F5012E5E2
:1037C7005A640160030238ABE546D39F50030238C1
:1037D700ABE55A7018C3E5459FF55D74602FF58218
:1037E700E4341EAD82F55E8D5F7F40801BE55AB4E1
:1037F7000119C3E5469FF55D74B02FF582E4341EC9
:10380700AF82F55E8F5F7F101200167FF47E011284
:103817006C387D207F051266707D1A7F08126670EE
:103827007FC87E00126C38E4F55BE55BC3955D509D
:1038370061055FE55FAE5E7002055E14F5828E83FB
:10384700E0F55C123A6038880038660A386A0B3847
:10385700700C38760D387C0E38820F0000388EE4F5
:10386700FD80277D5F7F0780227D5E7F06801C7D30
:103877000A7F0280167D327F0280107D467F02809C
:103887000A7D0A7F038004AD5CE4FF126670055B66
:103897008098E55A70047F408007E55AB401057F98
:0438A70010126EAEDF
:0138AB0022FA
:10507F00200E10754406901DB8E06003D20E22E496
:10508F00F54222E528D394004003152822C2CA1501
:10509F0044E54414603D14603214601D146015140F
:1050AF007049901DB8E0FF7003F54222122C4C900E
:1050BF001DB9802F901DBA8015901DBBE0FF7003A6
:1050CF00F54222122C4C901DBC8018901DBDE0FFA4
:1050DF00020026901DBEE0FF7003F54222122C4CF9
:1050EF00901DBFE0FF120026D2CA22E4F542C2CAC9
:0350FF00C20E22BC
:10661600900028E0FF6026200E07124D2E752814E4
:1066260022E528D394004003152822202708D2CA41
:0E663600752814D22722C2CA75287DC22722D9
:1065B800200E0C7F1C124D2E75286475793C22E53F
:1065C80028D394004003152822AF791579D3EF64B6
:0E65D800809480400475286422C20EE4F542CF
:0165E6002292
:1062F100E54214601C14601C14601F1460221460B9
:106301002224057021C2CAC20EC227C21DE4F5446F
:106311002202507F126616D21E22124166D21E221E
:076321000265B812510222CF
:1063FF00BF010790002A7418F022BF020790002AED
:10640F007412F022BF030590002A8014BF04079076
:10641F00002A740BF02290002ABF05047409F022A1
:04642F00740CF022D7
:024FF900AC0703
:104FFB00C3EC64809480404AEC64809488504320D6
:10500B002B21E4FD124D38C333CE33CED8F9124CDD
:10501B00B374102BF58274003AF583EFF00DBD08D5
:10502B00E3801FE4FD124D38C333CE33CED8F912D3
:10503B004CB374182BF58274003AF583EFF00DBD69
:10504B0008E3202B16E4FDEDFF3395E0FE74102FE3
:10505B00F5827400124CE4BD08ED22302B15E4FDF3
:10506B00EDFF3395E0FE74182FF5827400124CE4BB
:03507B00BD08ED80
:01507E00220F
:1053D7007D3F7F091266707D507F08126670906F5F
:1053E7002B12543E7D5B7F06126670906F2C125411
:1053F7003E906F2DE493FDE4FF126670906F2EE4EC
:105407009324BE601414601514601814601B146094
:105417001E240570217D0A80067D3280027D467F2D
:105427000280107D0A7F03800A7D287F0380047D28
:10543700467F0312667022E493FDE4FF1266702232
:105EFE008F5BE55B7005D22DFF8009E55BB4010772
:105F0E00D22D7F011259D07D4B7F021266707D0219
:105F1E00E4FF1266707D32E4FF1266701253D7E50D
:105F2E005B70028005E55BB401057F40126EAE2208
:103D3400A209300501B350307D017F04124EE950D1
:103D44002320050E30090B9000A4E0FF7C0B7D605E
:103D5400800F30050F20090C9000A5E0FF7C0B7D3F
:103D640080125BEFA2099205A20A300601B350301B
:103D74007D027F04124EE9502320060E300A0B9078
:103D840000A6E0FF7C0B7DA0800F30060F200A0CFC
:103D94009000A7E0FF7C0B7DC0125BEFA20A9206A5
:103DA400A20B300701B350307D037F04124EE9505B
:103DB4002320070E300B0B9000A8E0FF7C0B7DE066
:103DC400800F30070F200B0C9000A9E0FF7C0C7DC6
:103DD40000125BEFA20B9207A20D300801B3503022
:103DE4007D047F04124EE9502320080E300D0B9001
:103DF40000AAE0FF7C0C7D20800F30080F200D0C02
:103E04009000ABE0FF7C0C7D40125BEFA20D9208AA
:013E1400228B
:1064F800534103900024E0FE543FFF7804088001D4
:1065080023D8FD54F0FFEE30E40343070490002441
:0F651800E030E503430708EF4241C2AF124CD514
:016527002251
:02299A008F6B41
:10299C00302F05756CF48003756C64E56B64017005
:1029AC0029AF417803EF08800123D8FD3392307FA3
:1029BC001020300B122AB67F10126EEF022AAE12C4
:1029CC002AC17F10126F02022AAEE56B64027028D6
:1029DC00AF417802EF08800123D8FD3392307F207D
:1029EC0020300A122AB67F20126EEF8008122AC1FC
:1029FC007F20126F02022AAEE56B64037028AF4190
:102A0C007801EF08800123D8FD3392307F402030CD
:102A1C000A122ACC7F40126EEF8008122AD77F4010
:102A2C00126F02022AAEE56B6404701EE54133920C
:102A3C00307F8020300A122ACC7F80126EEF800803
:102A4C00122AD77F80126F028058E56B64057027BD
:102A5C00AF417805EF08800123D8FD3392307F0415
:102A6C0020300A122AE27F04126EEF8008122AED3F
:102A7C007F04126F02802BE56B6406702CAF4178DB
:102A8C0004EF08800123D8FD3392307F0820300AF0
:102A9C00122AE27F08126EEF8008122AED7F0812CC
:092AAC006F02AF6C7E00126C3861
:102AB50022126F02AF6C7E00126C3822126EEFAFDD
:102AC5006C7E00126C3822126F02AF6C7E00126CA5
:102AD5003822126EEFAF6C7E00126C3822126F0234
:102AE500AF6C7E00126C3822126EEFAF6C7E001256
:032AF5006C382218
:105D6200900024E030E0057F10126F02900024E0E2
:105D720030E1057F20126F02900024E030E2057FBF
:105D820040126F02900024E030E3057F80126F0220
:105D9200900024E030E4057F04126F02900024E0BA
:095DA20030E5057F08126F0222B2
:106CA40030030A124D19C203C211C21E2230040954
:0A6CB400124D19C204C213C21E22C1
:106528008F708D71E570B4011FE5717003125C8581
:10653800E571B401077880E6FF125A73E571B43249
:106548000E7FF47E01026C38AD71AF701266702256
:10667000EFFEEDFF1280008E2D8F2E125362757487
:1066800032AF741574EFD39400400EE4F573E573E4
:09669000C3943A50EC057380F547
:0166990022DE
:10536200D2A8AFA875A881C214852E82852D83E4A8
:1053720093C4540FFE4306F08E80C284D28500C2CD
:10538200870000D287007580FF7580FEC284C285C7
:1053920000C2870000D287007580FFD2147D407C56
:1053A2001FE4FE30B40D0EBE32F9ED1D70011CED8E
:1053B2004C70EE7C1F7D40E4FE20B40D0EBE32F92F
:1053C200ED1D70011CED4C70EE8FA8C2A87F0A7E05
:0453D20000126C3821
:0153D60022B4
:10669A007580FDC284C28500C28700000000D287CF
:1066AA00007580FF7F0A7E00126C387F997E09127E
:0A66BA0080008E2D8F2E12536222F5
:10422700D284D285C286A2809217A2819220A282CE
:104237009218A2839221D2862001537D027F011218
:104247004EE940137D037F01124EE9400A301707FC
:10425700301932D22480377D027F01124EE9500F88
:1042670030170C302009301904D224802180167DA4
:10427700037F01124EE9501220170330200C30192A
:1042870004D22480091267678004C219C22420025D
:104297004E7D027F02124EE940127D037F02124ECD
:1042A700E94009301806301B2FD225227D027F02F4
:1042B700124EE9500E30180B302108301B03D2255F
:1042C7002280157D037F02124EE9500F201803301C
:1042D7002109301B03D2252202678FC21BC2252268
:10676700753D1E753E60E4FFE53E2FF582E4353D3D
:10677700F583E4F00FBF50F0753D1E753E60E4F5FC
:0767870045C226C211D21920
:01678E0022E8
:10678F00753F1E7540B0E4FFE5402FF582E4353FBD
:10679F00F583E4F00FBF10F0753F1E7540B0E4F5C0
:0767AF0046C228C213D21BF1
:0167B60022C0
:106BE200C284D285C286A2809209A281920AA2821E
:0D6BF200920BA283920DD286D284D285220E
:10612700E57E2560F582E4357DF5832274FF123A1A
:1061370036E4FBFAF9F8C3023A23057F7480257E1B
:10614700F57EE4357DF57D22F582E4341DF5832265
:0B615700757F01757D00757E20E4223D
:1042E7007D027F07124EE950057F04126EEFC22947
:1042F700D223E4F5427FE87E03126C38C298C2AF3E
:10430700C2307F03122ED2755E7F755D96755C98FD
:10431700755B00785B126133504430983E1200069B
:10432700126E05EF14601824F0602624C1600B2478
:10433700F670287F06126F148021126211801C7F8D
:1043470006126F141269C01264F8125DF3D2298045
:104357000A7F06126F14125A23D2293029B5E4783E
:1043670085F6D2307F01122ED27F40120016C22F5F
:1043770012697A7D467F021266707D1E7F0712667C
:10438700707D147F081266707D327F03126670C2DB
:0D439700307F03122ED27FFF126EAEC223C4
:0143A40022F6
:105A2300126157F55F7F02126F14E57F2402F5615F
:105A3300AF7F126F14E4F560126127E0FF126F1459
:105A4300126127E02561F5610560E560C39480403C
:105A5300E7AF61126F147F03126F14126F1CEF64B0
:0F5A630015600C126141055FE55FC3942240B6E8
:015A72002211
:1069C000126157F55F1266ED50077F06126F148053
:1069D000057F15026F14126141055FE55FC39422C4
:0269E00040E392
:0169E2002292
:1066ED00E4F560126F1C74D0256012614FEFF00558
:1066FD0060E560C3948440EB126DE3901E52E0B5EB
:08670D000705126C53D322C3EF
:016715002261
:106C5300E4FF74D22FF582E4341DF583E0FEE57E74
:0A6C63002F12612BEEF00FBF7FE847
:016C6D002204
:106DE300E4FFFE74D02E12614FE02FFF0EBE82F33C
:016DF300227D
:10621100E4F55FF5657564E0756393756204F56196
:10622100786112613350213098F61200068F60E5D3
:106231006064046013AF65056574D02F12614FE58A
:0862410060F0255FF55F80D8D5
:016249002232
:04000600AF99C29854
:01000A0022D3
:086F14003099FDC2998F99220A
:076F1C003098FDAF99C29807
:016F2300224B
:106CF1000C0102030405060708090A0B0C01020333
:086D01000405060708090A0B4E
:10671600AF5FEF3395E0FE75F007EF123A54EE7572
:10672600F007A42583F583E0227883E6FF126CD870
:09673600EF22C295D297D2AF22E6
:10685300C22CC2AF126F247F83126D09126AF11228
:1068630067387884E66F600B125E7B302B05125F0E
:056873003E922CA22C56
:0168780022FD
:105F3E007984E778876660367884E6FF7887F6EFAF
:105F4E007013E552C3940A500C7D077F04124EE97C
:105F5E005003125E387D057F04124EE95010E54164
:105F6E0054036005123FC9D322123FC9C322C32274
:103FC900E4F55F900A50126716700302408D900A5B
:103FD9005112671D6016788166600302408D900A50
:103FE90052126716788866600302408DAF5FEF331F
:103FF90095E0FE900A5312671DFF7880E6FEEF6E8A
:104009006020EF601DB4080BEED394014005EE94D7
:1040190007400FEF6409706CEE64016005EE6407F8
:104029007062AF5FEF3395E0FE900A5412671DFF8F
:10403900F46006EF788366704BE55FFD3395E0FC2D
:10404900900A5575F007ED123A54EC1267257884F9
:10405900667031D201D20274BD2DF58274003CF52F
:1040690083E0FFC007EDAE047805C333CE33CED865
:10407900F92480F582740E3EAD82FCD007125BEF05
:10408900C201C202055FC3E55F64809493500302D5
:024099003FCC1A
:01409B002202
:105E38007D087F04124EE9500D7883E6FF126CD876
:105E4800EFC39407402CD2307F01122ED27F40122C
:105E58000016C22F12697AD201D202E4FD7F0A121B
:105E68004F71C201C2027F50126EAEC2307F011262
:035E78002ED22205
:105E7B00C2AF126F247FBF126D09126AF17884A62C
:105E8B0007126AF17884A607126AF17883A60712C3
:105E9B006AF17888A607126AF17881A607126AF16F
:105EAB007880A607126AF17882A607126F24126710
:025EBB0038228B
:1057BC00C2AF126F247F8E12580B7F90126D097F2F
:1057CC00A7126D09126F247FBE126D09E4FF126DD2
:1057DC00097884E6FF126D097883E6FF126D09786B
:1057EC0088E6FF126D097881E6FF126D097880E674
:1057FC00FF126D097882E6FF12580B1267382212DD
:0B580C006D09E4FF126D09126F2422E9
:105A73008F72E572B401047D63803EE572B4020661
:105A83007D087F068035E572B403067D317F08808B
:105A93002AE572B404067D617F08801FE572B405B0
:105AA300067D257F088014E572B406067D597F03C1
:0F5AB3008009E572B407077D487F0712667022ED
:026CD800AE0705
:106CDA00EE54F0FF780408800103D8FD75F00AA489
:066CEA00FFEE540F2FFF26
:016CF0002281
:105C850012672F906CF193FF1234C178841267313B
:105C9500601B7884126731C3940A50077D327F06F2
:105CA5001266707884E6FF126CD81234C112672F21
:105CB500C3940C50067D0A7F0280047D507F061236
:0A5CC50066707D507F0512667022A4
:10597A007FF47E01126C387D097F06126670788189
:10598A001259C07D0E7F031266707D357F0612663E
:10599A00707D097F0612667078881259C07D1E7F55
:1059AA00091266707D1E7F071266707882E6FF1202
:1059BA006CD81234C122E6FF126CD81234C17FF4BB
:0659CA007E01126C382280
:076F2400C2B6C295D295220E
:106D0900E4FEC297EF30E002D297C2B6D2B6EFC323
:066D190013FF0EBE08ECA2
:016D1F002251
:106AF100E4FFD297FED2B6C2B6A297E433C43333D1
:0F6B0100335480FDEFC313FFED42070EBE08E6CD
:016B10002262
:10570400EF3395E0FE74702FF58274003EF583E06C
:10571400FF22AF5AEF3395E0FEEF222460F5827446
:10572400013EAD82FCD22922900520E0F547A3E09A
:10573400F548222450F58274053EAD82FC22900087
:10574400BAE0FF7C0E7D2022D222D201E4FF22C2E5
:0D57540001C2227F1922D222D2307F022210
:10283900E5527008126ED88F52022934E552B40558
:10284900081243A58F52022934E552B40B08126CC1
:102859006E8F52022934E552B40A08125CCF8F52A6
:10286900022934E552B40F081260378F5202293415
:10287900E552B414081223528F52022934E552B496
:102889001908126B4E8F52022934E552B41E0812F0
:102899006A298F52022934E552B42308126A8F8FAC
:1028A90052022934E552B42807126EBC8F52807B3C
:1028B900E552B42D071267DF8F52806FE552B432AB
:1028C9000712624A8F528063E552B43E07126B6C5D
:1028D9008F528057E552B43C07126DAD8F52804B31
:1028E900E552B43307126A6D8F52803FE552B44105
:1028F90007126E368F528033E552B44C07126E467A
:102909008F528027E552B44407126E568F52801BAE
:10291900E552B437071258718F52800FE552B43916
:10292900071258178F528003E4F552E553700612C7
:10293900000E8F5322E553B40506126F0B8F5322F5
:10294900E553B40A06126E668F5322E553B40F0697
:10295900126E758F5322E553B41406123B708F53D0
:1029690022E553B43D06126B8A8F5322E553B43FD7
:10297900061265588F5322E553B443061267B78F81
:102989005322E553B44D06126AB08F5322E4F5532E
:01299900221B
:0D6ED80090052AE0F52BA3E0F52C7F0522A4
:1043A500302414201011C21C7D047F01124EE950E7
:1043B500037F0B227F0A227F0812632850061246CC
:1043C500877F0022202408301005C2107F05227D3A
:1043D500057F06124EE9501EE539453870189000E4
:1043E500B5E0FF7C0D7D80125BEF90052EE0F53882
:1043F500A3E0F53980557D067F06124EE9501EE58E
:104405003C453B70189000B6E0FF7C0D7DA0125B2B
:10441500EF900530E0F53BA3E0F53C802E7D077F6E
:1044250005124EE9500D30000AE52C452B7004C2EB
:10443500008018300F0AE52C452B7004C20F800B45
:104445007885E6B405057F04125180E5517008753D
:0A445500510AD22B1268537F052292
:106C6E00200F1590053BE0F54E2024037F0522E50D
:0B6C7E004ED3940050F3D20F7F0A2287
:105CCF007D077F05124EE9500C7D077F05124EE9C7
:105CDF00503230002F7D017F01124EE95026D23015
:105CEF007F01122ED27F011200167D027F07124E06
:105CFF00E950057F04126F029000A0E0FF7C0A7D3F
:0A5D0F00E0125BEF12572C7F0F2209
:10603700302437E5484547700C7D087F01124EE94B
:1060470050037F372230030EE53A700A126CA47FA3
:106057000112001680113026037F14227885E6B4DA
:0D60670005057F031251807F0F227F142258
:1023520090053DE0F54B7F01126EAE126CA47D023A
:102362007F07124EE95009E54B70057F04126EEFAC
:102372009000A1E0FF7C0B7D00125BEFD22B126874
:1023820053E545700302247C7C017D001224FA503F
:10239200037F3E227C017D501224DA50037F3C22CF
:1023A2007C017D581224DA50037F3C227C017D108F
:1023B2001224E250081224EA50037F33227C017D6A
:1023C200201224E2500B9000BBE0FF7C0E7D408087
:1023D200207C017D281224F2500512574280127C83
:1023E200017D301224F250129000B9E0FF7C0E7D84
:1023F20000125BEF1267677F00227C017D40D229C9
:10240200E4FF1247E7500C7D067F04124EE95003A9
:102412007F4C227C017D381224FA50037F44227CB7
:10242200017D18C229E4FF1247E7500C7D057F01A8
:10243200124EE950037F4122E4F55A1257167803EF
:10244200C333CE33CED8F912571FE4FF1247E750F9
:102452001BAF5A125704C0071257167805C333CE62
:1024620033CED8F9125737D007125BA4055AC3E509
:102472005A648094A840C47F19221224EA500C7D29
:10248200077F05124EE9504130003E7885E6700420
:102492007F0180087885E6B404077F0212518080AC
:1024A200257D037F06124EE9501CE55745567016EE
:1024B2009000AFE0FF7C0C7DC0125BEF900532E034
:1024C200F556A3E0F5577F19227D077F05124EE9E5
:0724D20050052000027F0508
:1024D90022D229E4FF1247E722D229E4FF1247E773
:1024E900227D077F05124EE922D229E4FF1247E730
:0924F90022C229E4FF1247E72288
:106B4E003026031267677D077F05124EE950062037
:0E6B5E0000037F0522900538E0F54E7F1E22D1
:106A2900E54E70037F23227D027F07124EE950094C
:106A3900E54B70057F04126EEF3024037F0A227F35
:026A49001E220B
:106A8F0012572C7D067F01124EE9500C9000ACE09E
:106A9F00FF7C0C7D60125BEF900539E0F54E7F2D8A
:016AAF0022C4
:0E6EBC007FA0126EAE900539E0F54E7F2D22BC
:1067DF00D22B1268537D027F07124EE95009E54B09
:1067EF0070057F04126EEFE54E70037F3222302466
:0767FF00037F0A227F2D2217
:10624A00301E037F32227D047F06124EE9501FE57D
:10625A0055455470199000B0E0FF7C0C7DE0125B4C
:10626A00EF900534E0F554A3E0F5557F3222C230B1
:08627A007F01122ED27F0022E9
:106DAD0020220CD222E4FF12055BC2227F00227F3B
:026DBD003C2276
:106B6C00202218D2227F40120016D201121D99C287
:0E6B7C00017F40126EAEC2227F19227F3E22A0
:106E360020220A12574C1237B5125753227F41228D
:106E460020220A12574C1260B0125753227F442256
:106E560020220A12574C1254B3125753227F44224F
:05000E0000007F052247
:096F0B003025037F0A227F0522D4
:0F6E66009000A2E0FF7C0B7D20125BEF7F0F22DC
:0F6E75003025093028037F14227F0F227F14223B
:103B70009000A3E0FF7C0B7D40125BEFE5467003F5
:103B8000023C487D017F03124EE950707C017D08A4
:103B9000C2297F011247E750037F3F227C017D50FD
:103BA000123C4B50037F3D227C017D58123C4B5010
:103BB000037F3D227C017D40D2297F011247E750DF
:103BC0000C7D067F04124EE950037F4D227C017D5F
:103BD00028D2297F011247E75009125742125BEFA2
:103BE0007F00227C017D18C2297F011247E7500C1B
:103BF0007D057F02124EE950037F43227D027F0341
:103C0000124EE95043E4F55AAF5A1257187803C3DD
:103C100033CE33CED8F912571F7F011247E7501D1C
:103C2000AF5A125704C007AF5A1257187805C3335A
:103C3000CE33CED8F9125737D007125BA4055AC33A
:0A3C4000E55A648094A840C07F009C
:093C4A0022D2297F011247E72272
:106B8A00202218D222C2307F01122ED27F01126E29
:0E6B9A00AE7F0112055BC2227F00227F3D22EA
:1065580020222A12575A122ED27FF47E01126C384A
:106568007F10120016D202121B98C2027F10126E00
:10657800AEC2307F02122ED2C2227F00227F3F227B
:1067B70020222212575A122ED27FF47E01126C38F1
:1067C700D2027F011237B5C202C2307F02122ED227
:0867D700C2227F00227F432251
:106AB00020221B12575A122ED2D2027F011260B02E
:106AC000C202C2307F02122ED2C2227F00227F4D2C
:016AD00022A3
:1055E700AF5AEF3395E0FE22900520E0F547A3E0A0
:1055F700F54822900522E0F549A3E0F54A22246008
:10560700F58274013EAD82FCD2292274702FF58297
:1056170074003EF583E0FF22C202C2227F192224D2
:1056270050F58274053EAD82FC22055AC3E55A64E3
:105637008094A822D222C2307F0122D222C2307F98
:0256470002223D
:10326D00E5527006126A4B8F5222E552B4050612D2
:10327D0035C08F5222E552B40B061268068F5222CA
:10328D00E552B40A0612445F8F5222E552B40F067E
:10329D00126DBF8F5222E552B411061259228F5270
:1032AD0022E552B412061251FA8F5222E552B4148D
:1032BD0006120D448F5222E552B419061265E78F9E
:1032CD005222E552B41E061265888F5222E552B481
:1032DD002306125EBD8F5222E552B42806126ECA25
:1032ED008F5222E552B42D061261628F5222E552A1
:1032FD00B432061262828F5222E552B43C06126D30
:10330D00D18F5222E552B43D06126C898F5222E5BF
:10331D0052B43E061268E88F5222E552B43F0612AF
:10332D006DF48F5222E552B44106126B118F522269
:10333D00E552B443061269E38F5222E552B44C06AE
:10334D00126CBE8F5222E552B44D06126A068F5290
:10335D0022E552B437061258718F5222E552B43914
:10336D00061258178F5222E552B4380612690D8F86
:10337D005222E552B43306126A6D8F5222E552B4D1
:0C338D004406126D208F5222E4F55222FB
:106A4B0090052AE0F52BA3E0F52C7D067F02124E74
:106A5B00E9500C90052CE0F529A3E0F52AD21F7F15
:026A6B00052202
:1035C000302414201011C21C7D047F01124EE950DA
:1035D000037F0B227F0A22302514201211D21C7D7A
:1035E000047F02124EE950037F0B227F0A227F08DC
:1035F00012632850061246877F00222024083010CC
:1036000005C2107F0522202508301205C2127F0551
:10361000227D057F06124EE9501EE53945387018A7
:103620009000B5E0FF7C0D7D80125BEF90052EE0F1
:10363000F538A3E0F53980757D067F06124EE95016
:103640001EE53C453B70189000B6E0FF7C0D7DA068
:10365000125BEF900530E0F53BA3E0F53C804E7D3A
:10366000077F05124EE9500D30000AE52C452B70FE
:1036700004C200800B300F08E52C452B7002C20FEE
:103680007D067F02124EE95019301F16E52A4529A2
:103690007010C21F9000BCE0FF7C0E7D60125BEFDB
:1036A000800B7885E6B405057F04125180E55170E2
:0C36B0000875510AD22B1268537F0522C6
:10680600200F2190053BE0F54E202406201C037F37
:106816000522202506301C037F0522E54ED3940071
:0768260050E7D20F7F0A22A8
:10445F007D077F05124EE950127D077F05124EE949
:10446F004003024510200003024510201C3FD230AC
:10447F007F03122ED27F0F126EAE90000FE0B402A8
:10448F00047F05800990000FE0B403057F0112003F
:10449F00161255EF7D027F07124EE950057F041269
:1044AF006F029000A0E0FF7C0A7DE0804E301C512F
:1044BF0090000FE0FF64026005EF640370437F0F0D
:1044CF00126EAE7F05126328400BD2307F01122E81
:1044DF00D27F028009D2307F03122ED27F0A1200C0
:1044EF00167D027F07124EE950057F04126F0212EC
:1044FF0055FA9000A2E0FF7C0B7D20125BEF7F0F3F
:0A450F00221255EF1255FA7F0F2219
:106DBF00201C063024037F1122301C053025027F52
:026DCF0012228E
:10592200302452E5484547700C7D087F01124EE94C
:1059320050037F3722300329E53A70257FA0126E8B
:10594200AE90000FE0B401047F01800990000FE0E7
:10595200B402057F05120016E4F542C21EC203809E
:10596200113026037F14227885E6B405057F0312E1
:0859720051807F11227F1422F5
:1051FA00301C1030240D20100A7F0A126EAEC21C19
:10520A007F0A22301C4C30254920124630030312F3
:10521A006CA4E54A4549700C7D087F02124EE9509C
:10522A00037F3822300417E53A70137FA0126EAE5E
:10523A007F02120016E4F542C21EC2048011302811
:10524A00037F14227885E6B405057F031251807F17
:10525A001222201C1230250F20120CD21CC2307FC1
:0A526A0002122ED27F0A227F1422C6
:100D440090053DE0F54B7F0F126EAE201C0C900019
:100D5400A1E0FF7C0B7D00125BEF301C0C9000A324
:100D6400E0FF7C0B7D40125BEFE542B403037F148C
:100D740022126CA4E4F5427D027F07124EE9500969
:100D8400E54B70057F04126EEFD22B126853301CB2
:100D940003020E87E5457003020E877C017D001275
:100DA400100450037F3E227C017D50120FD4500367
:100DB4007F3C227C017D58120FD450037F3C227C5F
:100DC400017D10120FDC5008120FEC50037F332208
:100DD4007C017D20120FDC5003020EEE7C017D2885
:100DE400120FF4500C9000BAE0FF7C0E7D20020E2E
:100DF400F77C017D30120FF4500C9000B9E0FF7CB9
:100E04000E7D00020EF77C017D40D229E4FF1247DB
:100E1400E7500C7D067F04124EE950037F4C227C80
:100E2400017D3812100450037F44227C017D18C2D6
:100E340029E4FF1247E7500C7D057F01124EE9506B
:100E4400037F4122E4F55A1255E7EF7803C333CE0A
:100E540033CED8F9125605E4FF1247E7501D125558
:100E6400E7125612C0071255E7EF7805C333CE33A5
:100E7400CED8F9125626D007125BA412563140C7B9
:100E84007F1922201C03020F7AE5467003020F7AB1
:100E94007D017F03124EE94003020F327C017D087D
:100EA400C2297F011247E7500F7F50120016D2303B
:100EB4007F02122ED27F3F227C017D50120FE4501C
:100EC400037F3D227C017D58120FE450037F3D22B5
:100ED4007C017D10120FFC5008120FEC50037F337D
:100EE400227C017D20120FFC50129000BBE0FF7C9D
:100EF4000E7D40125BEF1267677F00227C017D400C
:100F0400D2297F011247E7500C7D067F04124EE977
:100F140050037F4D227C017D18C2297F011247E7CF
:100F2400500C7D057F02124EE950037F43227D025F
:100F34007F03124EE9503CE4F55A1255E7EF78036B
:100F4400C333CE33CED8F91256057F011247E7508A
:100F54001D1255E7125612C0071255E7EF7805C364
:100F640033CE33CED8F9125626D007125BA41256CC
:100F74003140C77F192212100C500812100C504136
:100F840030003E7885E670047F0180087885E6B4F9
:100F940004077F0212518080257D037F06124EE9EB
:100FA400501CE557455670169000AFE0FF7C0C7D51
:100FB400C0125BEF900532E0F556A3E0F5577F19B8
:0F0FC400227D077F05124EE950052000027F05B0
:100FD30022D229E4FF1247E722D229E4FF1247E78E
:100FE30022D2297F011247E7227D077F05124EE9AE
:100FF30022D229E4FF1247E722D2297F011247E7D1
:1010030022C229E4FF1247E7227D077F05124EE93A
:0110130022BA
:1065E700C219C2307F02122ED23026051267678089
:1065F7000630280312678F7D077F05124EE9500684
:0F6607002000037F0522900538E0F54E7F1E220C
:10658800E54E70037F23227D027F07124EE95009F2
:10659800E54B70057F04126EEF3024062010037F50
:1065A8000A22302508201205D21C7F0A227F1E22CB
:105EBD00201C051255EF80031255FA7D067F011245
:105ECD004EE95024E5427020201C0B9000ACE0FF01
:105EDD007C0C7D60800C301C0C9000ADE0FF7C0CC8
:105EED007D80125BEF7F2822900539E0F54E7F2DE6
:015EFD002282
:0E6ECA007FA0126EAE900539E0F54E7F2D22AE
:10616200D22B1268537D027F07124EE95009E54B8C
:1061720070057F04126EEFE54E601D30240620107C
:10618200037F0A2290000FE0640160093025062097
:0B61920012037F05227F2D227F3222A6
:10628200301E037F32227D047F06124EE9501FE545
:1062920055455470199000B0E0FF7C0C7DE0125B14
:1062A200EF900534E0F554A3E0F5557F3222C23079
:0862B2007F01122ED27F0022B1
:106DD10020220CD222E4FF12055BC2227F00227F17
:026DE1003C2252
:1068E80020221FC2307F02122ED2D2227F401200F5
:1068F80016D201121D99C2017F40126EAEC2227FCC
:0569080019227F3E2270
:106DF40020220BD222D202121B9812561F227F3F4E
:016E0400226B
:106C890020221512563B122ED27F40126EAE7F0182
:0B6C990012055BC2227F00227F3D221B
:106B1100202219125642122ED27F10126EAED201CD
:0F6B2100E4FF1237B5C201C2227F19227F412241
:1069E30020221D12563B122ED27F40126EAED230A1
:1069F3007F02122ED2D2027F011237B512561F2206
:036A03007F4322AC
:106CBE00202214125642122ED2D201E4FF1260B0DC
:0A6CCE00C201C2227F19227F412279
:106A060020221D12563B122ED27F40126EAED2307D
:106A16007F02122ED2D2027F011260B012561F22BE
:036A26007F432289
:106D2000202211125642122ED2D202E4FF1254B384
:076D300012561F227F4422CE
:10587100D2107D027F07124EE950057F04126EEFB0
:1058810090000FE0FF64016004EFB4030E7F01128A
:105891006EAE7F401258BA7F01801390000FE0B4C2
:1058A100020F7F05126EAE7F501258BA7F03126E3F
:1058B100EF7F50126EAE7F3922120016C22F12698D
:0958C1007AE4FD7F07124F712209
:105817003024037F3922E47885F6C21090000FE028
:10582700FF64016004EFB4030E7F01126F027F4033
:105837001258617F01801890000FE0B402147F03B3
:10584700126F027F05126EAE7F501258617F0312EE
:105857006EEF7F50126EAE7F0022120016C22F121B
:0A586700697AE4FD7F08124F7122F8
:10690D00D2127F0A126EAE7F40120016D22F12697C
:10691D007AE4FD7F07124F717F03126EEF7F5012E5
:05692D006EAE7F0022A8
:106A6D0030000B9000B8E0FF7C0D7DE0800C200025
:106A7D000E9000B7E0FF7C0D7DC0125BEFB2007F82
:026A8D001922CC
:1060B0008F5AE55A24FF922F12697AE55A70127F9F
:1060C00040120016D201E4FD7F09124F71C2018017
:1060D00015E55AB401107F10120016D202E4FD7FBC
:0C60E00009124F71C2027F50126EAE22F6
:104D4200C201C202D20C7F50126EAE7F80120016D8
:104D520075420390000FE0B401163024647F011203
:104D62000016302407E542D3940050F67F01804EAE
:104D720090000FE0FF64026005EF6403704330248B
:104D8200267F02126EAED2307F03122ED27F051220
:104D92000016302407E542D3940050F6C2307F0259
:104DA200122ED27F0580173025177F02120016308F
:104DB200250AE542D3940040033024F37F02126EA9
:0F4DC200AEE542708E7FA0126EAEC20CC21E22F2
:03000000026BFF91
:106BFF00758E0078FEE4F6D8FD9000007FFF7E1FB3
:0D6C0F00E4F0A3DFFCDEFA758188024C235F
:10399A00C2D530F707B2D563F0FF05F030E70CB2B5
:1039AA00D5F4048463F0FF05F080018430D502F475
:0239BA000422E5
:1039BC00EF8DF0A4A8F0CF8CF0A428CE8DF0A42E1F
:0239CC00FE22D9
:1039CE00BC000BBE0029EF8DF084FFADF022E4CCDD
:1039DE00F875F008EF2FFFEE33FEEC33FCEE9DECA6
:1039EE00984005FCEE9DFE0FD5F0E9E4CEFD22EDEC
:1039FE00F8F5F0EE8420D21CFEADF075F008EF2F36
:103A0E00FFED33FD4007985006D5F0F222C398FD26
:053A1E000FD5F0EA22C3
:103A2300EB9FF5F0EA9E42F0E99D42F0E89C45F0F9
:013A33002270
:103A34007401FF3395E0FEFDFC080808E6CF2FF67D
:103A440018E6CE3EF618E6CD3DF618E6CC3CF62256
:0C3A5400A42582F582E5F03583F583227D
:103A6000D083D082F8E4937012740193700DA3A3F5
:103A700093F8740193F5828883E473740293686009
:063A8000EFA3A3A380DF09
:106E0500EFC39461400AEF947B5005EF24E0FF2225
:016E1500225A
:00000001FF
